:03000000020257A2
:060003007F011241E02222
:03000B0002466545
:10000E00CD30E11520E00FC083C08288828C83CD75
:0C001E00F0D082D08322CDF222CDF62259
:10002A00CB30E11520E00FC083C08289828A83CB5E
:0C003A00F0D082D08322CBF322CBF7223F
:10004600ED30E11320E00EC083C08288828C83E00D
:10005600D082D08322E2226405700EC083C08288DB
:0B006600828C8393D082D08322E6229C
:10007100EB30E11320E00EC083C08289828A83E0E5
:10008100D082D08322E3226405700EC083C08289AE
:0B009100828A8393D082D08322E72272
:10009C0088F0A8817404C0E0C0F018E6C0E008E65F
:1000AC00C0E00886F018188001A3E0C608D5F0F966
:0200BC00F82228
:1000BE00EEC0E0EFC0E088F0E58124FDF8ECC6C0AC
:0900CE00E008EDC6C0E0A8F02234
:0C00D700E0A3FCE0A3FDE0A3FEE0FF229C
:0C00E300ECF0A3EDF0A3EEF0A3EFF02290
:1000EF0075F004AA83AB82D083D082E493A3CAC5F0
:1000FF0083CACBC582CBF0A3CAC583CACBC582CB7B
:08010F00D5F0E8C082C0832294
:10011700E5F06010C3EC13FCED13FDEE13FEEF13D7
:05012700FFD5F0F022FD
:10012C00120235C380021819E637F6DAF9020226F4
:10013C00E0A3FEE0FFEF8DF0A4CFC5F0CCA42CFC27
:09014C00EE60038DF0A42CFE22EC
:10015500C2D1C2D5EE30E707D2D1D2D5120202EC18
:1001650030E705B2D112020A12017D30D103120225
:100175000230D50312020A22BC000EBE0032EF8DFA
:10018500F08420D226FFADF0227B0075F008EF2F1A
:10019500FFEE33FEEB33FBEE9DEB9C4005FBEE9D46
:1001A500FE0FD5F0E9E4CECDCBCC227EFF7FFF223A
:1001B500EDB410005022EE8DF084FEEF54F045F0C2
:1001C500C48DF084C4FCEF540FC445F0C48DF08495
:1001D500FFADF0E4CC4FFF22EE8DF08420D2CC7E33
:1001E50008CEC5F0CDCBEF2FFFED33FD10D7079B24
:1001F5005005D5F0F1229BFD0FD5F0EA22C3E49F0F
:0D020500FFE49EFE22C3E49DFDE49CFC226C
:0C021200EE30E707E4C39FFFE49EFE22ED
:10021E0074F9800674FA800274FCD083D082258132
:07022E00F581C082C08322AC
:0F023500E5D054182407F8E58124FCF97A042257
:10024400EFB40A077F0D1202447F0A3099FDC29968
:030254008F99225D
:0F025700758124E4787FF6D8FD75A0FF02497306
:08026600C204750A0112000335
:10026E001243218F0BE50B146008146016146025E1
:02027E008031CD
:10028000E50AB40101D34004150A8025750A0680E9
:0602900020E50AB406049B
:04029600120003222D
:10029A00AF0A121D4130040F22E50AB406005004C9
:1002AA00050A8003750A01E50AB40403020407502B
:1002BA0014E50A14602014700302035F1470030229
:1002CA0003C20205E7E50A24FB700302044C14701A
:0602DA00030204B9808E4E
:1002E0007B027A0079007D057C15786912081D7FF4
:1002F000017B027A007900124293900106E0700BB4
:100300007F027B057A15797A124293900106E0FA12
:10031000B4010B7F027B057A15798B124293900111
:1003200006E0FAB4020B7F027B057A15799C124233
:1003300093900106E0FAB4030B7F027B057A1579EE
:10034000AD124293900106E0FAB404028003020564
:10035000E77F027B057A1579BE12429302026E7B1B
:10036000027A0079007D057C1578CF12081D7F0187
:100370007B027A0079001242939000FDE0600790C2
:10038000010CE0B401117B027A0079007D057C1537
:1003900078E012081D801D9000FDE0FDE4C0E0C083
:1003A000057B027A0079007D057C1578F112081D25
:1003B000158115817F027B027A0079001242930237
:1003C000026E7B027A0079007D057C1678031208A4
:1003D0001D7F017B027A0079001242939000FBE0BE
:1003E000C0E0A3E0C0E07B027A0079007D057C16C6
:1003F000781412081D158115817F027B027A00791D
:100400000012429302026E7B027A0079007D057C25
:1004100016782412081D7F017B027A0079001242AF
:1004200093900102E0C0E0A3E0C0E07B027A007993
:10043000007D057C16783512081D158115817F0217
:100440007B027A00790012429302026E900106E06C
:0E045000FA64026009EA64036004EAB4041668
:10045E00E50BB40102150AE50BB403028003020595
:10046E00E7050A02026E7B027A0079007D057C1692
:10047E00784512081D7F017B027A007900124293A3
:10048E00900104E0C0E0A3E0C0E07B027A007900B6
:10049E007D057C16783512081D158115817F027B2E
:1004AE00027A00790012429302026E7B027A007980
:1004BE00007D057C16785612081D7F017B027A009E
:1004CE007900124293900106E0601514603E1460AC
:1004DE006714700302057114700302059C0205C5B2
:1004EE009000FBE0C0E0A3E0C0E09000FDE0FDE482
:1004FE00C0E0C0057B027A0079007D057C16786726
:10050E0012081D74FC2581F5810205C59000FBE0E3
:10051E00C0E0A3E0C0E09000FDE0FDE4C0E0C00557
:10052E007B027A0079007D057C16787812081D749E
:10053E00FC2581F5810205C59000FBE0C0E0A3E03B
:10054E00C0E09000FDE0FDE4C0E0C0057B027A0053
:10055E0079007D057C16788912081D74FC2581F5BD
:10056E008180549000FBE0C0E0A3E0C0E09000FD6D
:10057E00E0FDE4C0E0C0057B027A0079007D057CD9
:10058E0016789B12081D74FC2581F5818029900038
:10059E00FBE0C0E0A3E0C0E09000FDE0FDE4C0E0C1
:1005AE00C0057B027A0079007D057C1678AD1208B5
:1005BE001D74FC2581F5819000FDE0600790010C13
:0405CE00E0B4010A8A
:1005D2007420900005F07441A3F07F027B027A0040
:0805E200790012429302026E3F
:0605EA00750A0112000376
:1005F0001243218F0BE50B1460081460161460671A
:02060000807305
:10060200E50AB40101D34004150A8067750A058022
:0606120062E50AB40504D4
:0406180012000322A7
:07061C00900111E0B401118F
:10062300AF0A1223921243218F0BE4F50B300432ED
:0106330022A4
:100634001200037F017B057A1979C91242937F0264
:100644007B057A1979DA12429312430EE4FE7FFA9B
:100654001242F612430E7E077FD01242F6120003B6
:1006640022800EE50AB405005004050A8003750AC9
:1006740001E50A14600E14601C14602A1460381416
:0406840060468053F9
:100688007B027A00795E7D057C1978EB12081D8063
:10069800427B027A00795E7D057C1978FC12081D80
:1006A80080317B027A00795E7D057C1A780D12080C
:1006B8001D80207B027A00795E7D057C1A781E12E7
:1006C800081D800F7B027A00795E7D057C1A782FE1
:1006D80012081D740690005EF07F017B027A007993
:1006E8005E1242937B027A00795E7D057C1A78401F
:1006F80012081D7405900062F004A3F07F027B02CB
:0A0708007A00795E1242930205F0B8
:06071200E4F508120003EB
:100718001243218F09E50914600814601614604219
:02072800804E01
:10072A00E508B40001D34004150880427508038027
:10073A003DE508600B14601014601714601C802ECD
:10074A0012026612000380261205EA120003300420
:10075A000D22122EF9120003801412000322800EB9
:10076A00E508B40300500405088003E4F508E50829
:0D077A00600B146019146027146035804274
:100787007B027A0079867D057C1B786112081D80C3
:10079700317B027A0079867D057C1B787212081DF1
:1007A70080207B027A0079867D057C1B788312087E
:1007B7001D800F7B027A0079867D057C1B78941259
:1007C700081D7406900086F07F017B027A00798607
:1007D7001242937B027A0079867D057C1A78401253
:1007E700081D740590008AF004A3F07F027B027A4B
:0907F700007986124293020718F2
:10080000A881058118EBC6C908CAC6CA08F67BFFCD
:10081000112ED0E0D0E0D0E0C082C08322D083D0BF
:1008200082EDC0E0ECC0E0E8C0E0C082C083E581BA
:10083000F82425F58108E8C9CBF709EAF709EBF7B1
:1008400009770009E924F6FA75F000C2D5E924FC1D
:10085000F8E924F9F9ECC0E0E8C0E0D1E51200467F
:10086000FFE92409F9D0E0F8D0E0FCEF605020D592
:1008700074B4250AE4FB74FFFCF7D2D580D3D1FE13
:1008800080CFFF20F71CBCFF067014D2F380C2ECAF
:10089000C0F075F00AA42FD0F030F703F78001FC08
:1008A00080AFB7FF03EF80F4E780E57F00D1FE194A
:1008B0001709800DEF24D0B40A0040C68093B6FF1C
:1008C000EAE581C39421F581E4FED0E0FFD082D037
:1008D00083D0E004600ED083D0821581158115810C
:1008E000C082C08322900F78E49360256FA36006D6
:1008F000A350F5A380F293FF400442F080BEE4A32E
:10090000938F83F582E4C2D130F705B7FF027700F9
:100910007340A1D3A380D1EAC8FDE620F703FC8091
:1009200001F71A1AEDF88094D2D17F7880027F58AF
:10093000D17990100421CCBCFF05B7FF02805AC0CA
:10094000F08AF0EAC92420F583E8FEECC0E0D1E5A6
:10095000120046FF601AC583C9C583F70B19E9C5A4
:1009600083F908B800010CEE2404F9E7C39B70E09A
:10097000D0E0FCE5F024FDFAD0F08B82A98309EEEB
:10098000C394FBF583F805828004E7F60809D58255
:10099000F9A9831819C2F0414F8AF0EAC9F583E832
:1009A000FED1E5120046FF6013EEC8CE8D82D1FE67
:1009B000AD82EEC8CE08B800EA0C80E7A983E5F066
:1009C00024FDFA01487F30D179900806C2F7D18919
:1009D000E8CAC9C88049D2F7EA147D0230F4047D20
:1009E0000424FEF8E68A83A88330E70DD2D1C3E45D
:1009F00096F618DDFAA8838000C2F7D179900A052F
:100A0000D189C9C8CAC9B1FF8015D179E618188043
:100A100004D1797425C2F7F70BCAC9C8CAC2F0E776
:100A2000FDE924002BF8B6300318DBFABB00080BF5
:100A300008BD00031B8013BDFF02800EEDC39BFEAB
:100A40004008600674305192EDFBEB70020148ECF7
:100A5000046023D39B401F601DFE7D2020F13830B1
:100A6000F3027D3030F023BD3018518E18EF30E6A0
:100A700001187111804030F03F71110B30F6390BC5
:100A80008036EF71111E30F6011E518E8028EE6007
:100A900005ED08F6DEFC2230F00771110B30F6018F
:100AA0000BE9FF2420F9E6F71918DBFAEDF719DE58
:100AB000FCEFF92420F8CCCBEB700201481919E8BF
:100AC000C0E0E6FFD1E50909EFD16AD0E0F818DB14
:100AD000EE090901481A1AD181900F6CE6086002EC
:100AE0002406936023F7190B30E504E4A380F3EBAD
:100AF000C0E0743AF7E924FCF908901004D1891891
:100B0000D0E02405FBE92404C8CAC9E92420F88000
:100B1000AC08EFF68FF030F604743008F622619BD3
:100B2000C2F79159BFFF0261ADEF60F22481FF204F
:100B3000E73618040FD113EBC39F60124010FDFE7F
:100B40000BE89FF8742EC618C6DDFC18805DF4040F
:100B5000FD7E000DE824F9F880057430F6180BDDF1
:100B6000F9742EF60B188043F4FD7E070DBD0700C7
:100B70004016E9FD097430F709E9C39870F7EDF9FB
:100B800080087430F60E0B08DDF8742EF6080B0B97
:100B90007430F6D113E8C39BF88010E92420F87470
:100BA00030F618742EF6187B027E00B1AD414AC2B1
:100BB000F78002D2F79159BFFF0280F1BF000E7497
:100BC00030F618742EF6087E007B02800EEF24812A
:100BD000FF18742EC608C6EBFE1E0BD113E8C39B8C
:100BE000F8EFC0E0B1ADD113D0E0FFC0F0E8C39B97
:0E0BF000F8E730F704746580027445F618EFDC
:100BFE0020E704762B8004762DF4041875F00A8411
:100C0E002430F618E5F02430F6EB2404FBD0F0D1B6
:100C1E002918B1FF61ADC2F78002D2F7D2F2915915
:100C2E00BFFF0261ADE7B4FF037406F7BF7B004060
:100C3E0016EF248120E706C397600C500A74822FAA
:100C4E00C7C397F7020B2917020BBCD179ECC0E092
:100C5E00C0F018E63308E63392D5186033B4FF407F
:100C6E00E6C2E76009900FBCC2D17B078007900FE8
:100C7E00C3D2D17B06E493F709A3DBF97B0330D112
:100C8E000A742B30D502742DF70B09197C80A184C0
:100C9E00EAC0E074307A08F709DAFC097C81A17D9C
:100CAE00CAC0E0EA75F010A4CAABF075F04DA42BE3
:100CBE00FBE435F0FCEA2410FAEB34C5FBEC34D936
:100CCE00FCE6C2E7FF75F056A4F42411C5F0F43427
:100CDE00C58FF0A42AE5F03BE43CFBC0E0E9C0E0A0
:100CEE00E8C0E0EBC0E020E707800812112C801F5F
:100CFE00F404FB121411D0F0D0E0F8C0E0187583A4
:100D0E000418E6C0E008D583F930F7DF121288D058
:100D1E00E0F8D0E02408F9EED2E7CE33EF332482A8
:100D2E00FAECFBD0E0FCE4C3CB33CBCD33CDCE33EA
:100D3E00CE33DAF37A0875F00A8460062430F71998
:100D4E001A0CE5F02430F7198BF0740AA4FBAFF0FF
:100D5E008DF0740AA42FFDAFF050010F8EF0740ABF
:100D6E00A42FFE743035F0F719DADDE9240AF9D034
:100D7E00E0FAE9D39AFBECFF247FFFCAC9C824FD31
:100D8E00FAE9FD09EF046003120F2FEDF909EF04E4
:100D9E006003120F2FEDF9D0F0D0E0FC7B0722E7B5
:100DAE00B4FF027406700820F0010E8E838016C305
:100DBE009E400EF583603674300BF618D583FA809C
:100DCE002CF404F583C0E0E9C0E0E8C0E0F92B04A0
:100DDE00F8EEC0E0EFC0E009120F2DD583FAD0E097
:100DEE00FFD0E0FED0E0F8D0E0F9D0E0FD08D12948
:100DFE0018D2F07F2D20D10C7F2B20F5077F2020DD
:100E0E00F602C2F0228982E92420F98B83E6F719D3
:100E1E0018D583F9A982E92420F822E9F582240164
:100E2E00F98B8330F22A20F027C2F2E608B42E02A4
:100E3E00D2F2D583F6E8C39BF88B8330F210E6B47A
:100E4E003005081BD583F7B42E07081B8006D2F297
:100E5E00E6F70908D583F9E9F8A98222BDFF051244
:100E6E000244800312000E09071922E9CAC8E924B8
:100E7E0001F922E9CAC8E92420F922A2F492D5C0C8
:100E8E00F0E582FD30D50623F582FD181818E685AB
:100E9E0083F084F620D5047B0180027B0308E5F005
:100EAE00D6C6C48583F084C4C6C445F0C48583F019
:100EBE0084D6DBE9E5F024F6500730D10224202455
:100ECE0007243AF70920D509DDC3D0F01818AB82F4
:100EDE0022DDB8181880F3E7F819E7FC19E7FDBD15
:100EEE00FF0122090907B70004190719221919224F
:100EFE00CACDE8C0E0E9C0E0E6FB08E6FA08E6F98C
:100F0E00EFBBFF05120244800A06B600031806085E
:100F1E0012002A080618D0E0F9D0E0F8CDCA22E96E
:100F2E00FD1BE7B4350FEBFE600709E719F709DE85
:100F3E00F718EDF92240EF09C3E899601AE719B4E2
:100F4E002E04F70980F104B43A067430F70980E7ED
:100F5E00F709E899FE80D1197431F70B80D4286E09
:100F6E00756C6C290049584450434C046C10620057
:100F7E00680023012D022B2020402E80002A091705
:100F8E006F09C578092858092E7309377509F96450
:100F9E0009D66909D6630A0A250A11700AD5660BA5
:100FAE0020650BB3450BAF670C28470C240020209F
:0B0FBE0020204E614E202020464E49AE
:100FC9001200D7EFB2E7FF80031200D7E58124FDB5
:100FD900F8F9E63308E63370060213B60213A504DE
:100FE90060FAEE33EF33700EE6FF18E6FE18E6FD01
:100FF90018E6FC0213B60460E3E58124FBF8D3ECA0
:101009009608ED9608EE9608EFC2E786F0C2F795C6
:10101900F0400FEFC6FF18EEC6FE18EDC6FD18EC3E
:10102900C6FC1213C7C3EB9FF5F0700EE58124FBD4
:10103900F9E4C3CC20D5730211049418605C400E06
:10104900E4FF19E7FE19E7FD19E7FC0210E0E4FFE8
:1010590030F405CEFCE4CDFF30F305E4CECDCCCFA2
:1010690030F21AE5D054184404F8EF54F0D6C4FF0E
:1010790008ECD6C4FC08EDD6C4FDEEC4FE740355D5
:10108900F06012F5F0C3EE13FEED13FDEC13FCEF67
:1010990013FFD5F0F030D55D8009E4CEFFE4FDFC07
:1010A90030D552C3E49FCC191919C797CD09C797F1
:1010B900CE09C797FF4E4D4C70140213B6DB0302DD
:1010C90013A9EC2CFCED33FDEE33FEEF33FFEF30CB
:1010D900E7EBECCFCECDFCEF30E70D0CBC00090DF2
:1010E900BD00050EBE00010BEB7005A2D102139DD8
:1010F900A2D10213B0E42FCC19191937CD0937CE73
:101109000937FF50090BEB700CA2D102139DEFCEEA
:10111900CDCCFF80C2EF13CE13CD13CC13FF80B714
:101129001200D7EF4E601AE58124FEF924FEF8E794
:1011390019477019EE33EF33B4FF030213A50213F5
:10114900A9E58124FDF8E63308E63380EB1213C7DD
:10115900248150082B5008A2D502139D2B50DFF78C
:10116900FAE61846197020B7800DEE33CAA2D513D6
:10117900FFCA13FE0213B6EC4D703CBE8046E6FC76
:1011890008E6FD08E680E4EC4D7039BE800280EE89
:10119900E4CEC7CDC6F5F008E4C6CCF9FBFFFA806A
:1011A90076E4CEC9E4CDCAE4FFCCFB803CE4C9CDEA
:1011B900CFCBECCACC8060E4F9FAFBFFCECDCCC52D
:1011C900F00880538CF0E660D8A4C5F0CDFAC5F0DC
:1011D900E6A42DCEF9C5F03400FDE6A42DC5F03402
:1011E90000FDCCFBC5F0CC7F0008E660C0A42EC58D
:1011F900F03C50010DCAFCC5F0CEE6A42AC5F03D6D
:1012090050010FC9FDC5F0CAE6A429C5F03F79010F
:10121900400119CBC5F0CF08E6A42AC5F03F500517
:101229000BBB000109CCC5F0FAE6A42CC5F03B5074
:101239000109CDC5F0CCE6A42DFDC5F039FE330872
:10124900500906B60011A2D502139DEA33FAEC3310
:10125900FCED33FDEE33FEEA30E7140CBC00100D53
:10126900BD000C0EBE000806B60004A2D580D9E662
:05127900A2D50213B034
:10127E00D083D0820213A91200D7EFC2E74E7003BB
:10128E000213A5C082C083E58124FBF8F9E6084667
:10129E0060DE1213C70FBF0006D083D08280E1EF4D
:1012AE0024805007C3CB9B500D80C5CB9B4007D0ED
:1012BE0083D08202139DF6F583EC4D701FBE801C09
:1012CE00E58124FBF8E583A2D513FFE692E7FE182D
:1012DE00E6FD18E6FCD083D0820213B6E58124FB2E
:1012EE00F8E6CEF618E6CDF618E6CCF6EFCCFFE82B
:1012FE002402F9F8E7FA19E7FB19E7FCE4F5F075B3
:10130E00821A758380801DE58303F58330E706A777
:10131E00F009E4F5F0C3EF33FFED33FDEE33FE409D
:10132E000C30E717C3EF9CED9BEE9A400EC3EF9C7B
:10133E00FFED9BFDEE9AFEE58342F0D582C9E7FAFA
:10134E0019E9F81919E720E7191ABA000302127EF3
:10135E00E5F025F0FFE633FC18E633FD18E633FE24
:10136E008009FE09E7FDE6FCE5F0FFEF30E7160C1D
:10137E00BC00120DBD000E0EBE000A0A7007D0830F
:0F138E00D08202139DEAA2D5D083D0820213B081
:10139D0074FF13FF7E80800774FF8001E4FFFEFD64
:1013AD00FC800613FFEE92E7FED0E0F8D0F0E58169
:1013BD0024FCF581C0F0E8C0E022E7D2E7C733098D
:1013CD00E733FB92D592D1EED2E7CE33EF33FF5018
:0413DD0002B2D52261
:1013E1003F8000003DCCCCCD3C23D70A3A83126F1D
:1013F10038D1B7173727C5AC358637BD33D6BF953A
:10140100322BCC7724E69595179ABE150A4FB11F5A
:10141100EB60105407700AEB543803241C12143C7F
:1014210022232312143CEB543870012203241CFBA9
:101431001200BEEB12143C12112C229013E1FC930A
:0E144100FF0CEC93FE0CEC93FD0CEC93FC22E4
:10144F001214958000EC3392D550031214837A2036
:10145F00C3EC20E712EF33FFEE33FEED33FDEC3339
:10146F00FC20E703DAEF22EA247DA2D513FFEC92EA
:10147F00E7CEFC22E4C39FFFE49EFEE49DFDE49CC7
:10148F00FC22C2D580C8EED2E7CE33EF3392D524FB
:10149F0081400CE4C2D5A2D513FC33FDFEFF2224FC
:1014AF00E0500474FF80EFF404FAE4CCCDCECF808B
:1014BF000DC3EF13FFEE13FEED13FDEC13FCDAF18A
:1014CF0020D507EECDFEEFCCFF22E4C39CFCE49DBC
:1014DF00FDE49EFEE49FCCFFEECDFE22EFC2E7FFC0
:1014EF0080A47A083392D5E4FDFEFF30D5031214A1
:1014FF0084EC334010EF33FFEE33FEED33FDEC336E
:10150F00FCDAEE80BEEA247EA2D513CC92E7CDCED4
:03151F00FF80B09A
:10152200E58124FEF88FF063F080E6F96480B5F07F
:101532001B188EF0E6B5F014188DF0E6B5F00D1814
:101542008CF0E6B5F006E4FFFE0213B68FF030F73A
:101552000689F030F701B340077F017E000213B61F
:0715620074FFFFFE0213B647
:101569004241545445525920545950452020202075
:10157900003A4E69434420202020202020202020AA
:1015890020003A4E694D482020202020202020208C
:101599002020003A4C69506F202020202020202054
:1015A900202020003A4C69494F4E2020202020203D
:1015B90020202020003A534C4120202020202020A8
:1015C90020202020200042415454455259204345AF
:1015D9004C4C20202020003A4155544F204445547A
:1015E90045435420202020003A2532642020202021
:1015F90020202020202020202000424154542E2049
:1016090043415041434954592020003A2534646DDF
:1016190041682020202020202020004348415247B3
:10162900452043555252454E542020003A253464F2
:101639006D412020202020202020200044495343B0
:10164900482E2043555252454E54202000455849B2
:1016590054204241545445525920202020004E69BB
:1016690043442025326443202534646D4168004E8B
:10167900694D482025326443202534646D41680052
:101689004C69506F202025316443202534646D4115
:1016990068004C69494F4E20253164432025346444
:1016A9006D416800534C4120202025316443202599
:1016B90034646D41680053455420424154544552A5
:1016C90059205459504500204E6943442020202078
:1016D9002020202020202000204E694D4820202055
:1016E900202020202020202000204C69506F20201D
:1016F90020202020202020202000204C69494F4E06
:10170900202020202020202020200020534C412070
:101719002020202020202020202020005345542054
:10172900424154544552592043454C4C00202532DE
:101739006420202020202020202020202020005349
:101749004554204341504143495459202020200009
:10175900202534646D41682020202020202020008D
:10176900202534646D4120202020202020202000C5
:101779004C4F41442046524F4D204C4F432E253269
:1017890064005341564520544F204C4F432E20208E
:10179900253264004552415345204441544120417A
:1017A9005420253264004C6F6164696E6720426180
:1017B9007474657279200046726F6D204C6F636195
:1017C90074696F6E2025326400204E6F2042617467
:1017D90074657279204461746100204174204C6FF2
:1017E900636174696F6E2025326420004F5645523B
:1017F900575249544520444154413F2000205361E8
:1018090076696E672042617474657279200020548C
:101819006F204C6F636174696F6E202532642000FC
:10182900455241534520444154413F202020202026
:101839000045726173696E672042617474657279DB
:1018490020002045584954204D454D4F52592020DC
:10185900202000204E69434420253264432025344A
:10186900646D416800204E694D482025326443204B
:101879002534646D416800204C69506F2020253162
:101889006443202534646D416800204C69494F4EFA
:101899002025316443202534646D41680020534C70
:1018A9004120202025316443202534646D4168009E
:1018B90020454D5054592020202020202020202030
:1018C900002020202020202020202020202020202F
:1018D9002000455241534520414C4C20444154413C
:1018E9003F200045726173696E6720416C6C20442A
:1018F9006174610020202046726F6D204D656D6F07
:1019090072792020005345542043454C4C532044C0
:10191900455445435400204155544F202020202050
:1019290020202020202000204D414E55414C2020D0
:101939002020202020202000534554204348415294
:10194900474552204D4F444500204359434C4520BB
:1019590043484152474520202000204348415247EF
:0B19690045204F4E4C5920202020004C
:1019740020444953434841524745204F4E4C592037
:101984000053455420434841524745204359434C52
:10199400450053455420534F554E4420564F4C5503
:1019A4004D4500204F4E20202020202020202020A4
:1019B40020202000204F46462020202020202020C8
:1019C4002020202000202043616E2774204163637F
:1019D400657373202000202053797374656D204D46
:1019E400656D6F72792000204C4F414420202020E7
:1019F40020534156452020002053415645202020A5
:101A04002020455241534520002045524153452052
:101A1400202020464F524D41540020464F524D4104
:101A2400542020204558495420200020455849542A
:101A340020202020204C4F41442020005573652055
:101A44003C3E20746F2053656C65637400204E6FB8
:101A540074204170706C696361626C652000466F2C
:101A6400722054686973204261747465727900202D
:101A7400466F722054686973204D6F64652020009E
:101A84002043454C4C5320444554454354494F4E00
:101A9400003A4155544F202020202020202020208F
:101AA40020003A4D414E55414C202020202020203A
:101AB4002020002043484152474552204D4F444581
:101AC400202020003A4359434C4520434841524783
:101AD40045202020003A434841524745204F4E4C70
:101AE4005920202020003A44495343484152474555
:101AF400204F4E4C59200020434841524745204333
:101B040059434C45202020003A4E6F742041707098
:101B14006C696361626C65200020534F554E44200C
:101B2400564F4C554D45202020003A4F4E20202042
:101B340020202020202020202020003A4F4646202C
:101B4400202020202020202020202000204558492B
:101B540054204F5054494F4E5320202000204241DE
:101B6400545445525920204D454D4F525900204D53
:101B7400454D4F525920204F5054494F4E53002049
:101B84004F5054494F4E532020202045584954006B
:101B9400204558495420202020424154544552594C
:101BA400002020534D41525420434841524745524E
:101BB4002000202053455256494345204D4F44456B
:101BC400202000202020204649524D5741524520D4
:101BD40020202000202056455253494F4E20312EBC
:101BE40030322020002043555252454E5420535445
:101BF4004550202020003A25346420202020202035
:101C0400202020202000204D41582E20564F4C5497
:101C14002F43454C4C20003A25352E326656202061
:101C2400202020202020202000204D494E2E205608
:101C34004F4C542F43454C4C2000204E45474154B3
:101C440049564520645620202020003A2532646DF0
:101C54005620202020202020202020202000205337
:101C64005550504C59204D4F4E49544F5220003A34
:101C740043482531642020202025352E32665673B2
:101C8400200020564F4C5441474520535445502082
:101C94002020003A2534642020202025352E326669
:101CA400562000204558495420534552564943452F
:101CB400202020005345542043555252454E542071
:101CC4005354455000534554204D41582E20562F0F
:101CD40043454C4C20003A25352E326656202020B0
:101CE40020202020202000534554204D494E2E20F2
:101CF400562F43454C4C2000534554204E454741F4
:101D04005449564520645620003A2532646D5620C5
:101D14002020202020202020202000534554205320
:101D24005550504C59204D4F4E2E200053455420B1
:0D1D3400564F4C5441474520535445500034
:051D41008F0C120003ED
:101D4600900106E0601214600F14606C1460691450
:081D56007003021DE1021E02F0
:101D5E009001077405F0A37478F07401900112F0ED
:101D6E00750D0A750E0F750FA09000FDE0FBE433A4
:101D7E00E4500114FCFD7E00AF03121454C004C0E5
:101D8E0005C006C007E4FCFD7496FE7444FF1211F4
:101D9E002CC004C005C006C0077CCD7DCC7E4C7F18
:101DAE003E12112C1214958E108F11751201804453
:101DBE009001077410F0A37468F07402900112F091
:101DCE00750D03750E0F750FA0E4F510F511751254
:101DDE000180219001077409F0A374C4F07402907D
:101DEE000112F0750D06750E1B750F58E4F510F502
:101DFE00117512031243218F13E50C14601B14701E
:101E0E00030220911470030220FF14700302222C8F
:091E1E001470030222EC021D46BF
:101E27007F017B057A1679BF124293E513B401153A
:101E3700900106E0B40001D34005E014F080067479
:0F1E470004900106F0E513B402028003021FF5B8
:101E56009000FBE0FAA3E0FB900102EAF0A3EBF0AE
:101E6600900102E0B40005A3E0B4640050099001BB
:101E760002E4F0A37464F0900102E0FEA3E0FFE444
:101E8600FC7D6412017DEE900102F0A3EFF090015B
:101E960002E0FEA3E0FFE4FC7D64120141EE900146
:101EA60002F0A3EFF0BE0B04BFB801D3400A9001C5
:101EB60002740BF0A374B8F07F051245868E148F5A
:101EC60015E4FCFD900116E0FEA3E0FF121491C09C
:101ED60004C005C006C00774CDFC14FDFE743DFFAA
:101EE60012112C8C168D178E188F19E4FCFDAE146A
:101EF600AF15121491C004C005C006C007AC16ADDC
:101F060017AE18AF19121288C004C005C006C00764
:101F16007466FEFCFD743FFF121522BF01028003AA
:031F2600021FEBAC
:101F2900900106E0600F14600C14604314604014C3
:051F39006077021FF1BA
:101F3E00E4FCFDAE14AF15121491C004C005C0062A
:101F4E00C007AC16AD17AE18AF19121288C004C078
:101F5E0005C006C0077455FEFCFD743FFF12112C20
:101F6E00121495EF9000FDF08079E4FCFDAE14AFF5
:101F7E0015121491C004C005C006C007AC16AD17EB
:101F8E00AE18AF19121288C004C005C006C0077C77
:101F9E00DD7D607E8A7F3E12112C121495EF90002B
:101FAE00FDF0803FE4FCFDAE14AF15121491C00499
:101FBE00C005C006C007AC16AD17AE18AF19121289
:101FCE0088C004C005C006C007E4FEFCFD743FFFD8
:0D1FDE0012112C121495EF9000FDF08006FA
:0F1FEB00E5129000FDF012430E22E513B403132C
:101FFA00900106E0B404005005E004F08005E49086
:10200A000106F0900106E0700F7B027A0079147DD8
:10201A00057C1678D012081D900106E0FAB4010F6B
:10202A007B027A0079147D057C1678E112081D90EE
:10203A000106E0FAB4020F7B027A0079147D057C6E
:10204A001678F212081D900106E0FAB4030F7B021B
:10205A007A0079147D057C17780312081D90010611
:10206A00E0B4040F7B027A0079147D057C1778149A
:10207A0012081D7406900014F07F027B027A007920
:10208A0014124293021D467F017B057A17792512A5
:10209A004293E513B401109000FDE0B51201D3405C
:0C20AA00069000FDE014F0E513B4020401
:1020B60012430E22E513B4030F9000FDE0B50D00A8
:1020C60050069000FDE004F09000FDE0FBE4C0E067
:1020D600C0037B027A0079147D057C1778361208D6
:1020E6001D158115817406900014F07F027B027A1B
:1020F600007914124293021D467F017B057A1779F7
:10210600481242939000FBE0FAA3E0BA0003B464DD
:102116000050099000FBE4F0A37464F09000FBE02B
:10212600FAA3E0FBEAB50E05EBB50F01D3400A9022
:1021360000FBE50EF0A3E50FF0E513B401209000D7
:10214600FBE0B40006A3E0B46401D340119000FCA8
:10215600E024CEFB9000FBE034FFF0A3EBF0E513A8
:03216600B4026E52
:102169009000FBE0FAA3E0FB900102EAF0A3EBF098
:10217900900102E0B40005A3E0B4640050099001A5
:1021890002E4F0A37464F0E4FCFD900102E0FEA314
:10219900E0FF121491C004C005C006C0077C0A7D87
:1021A900D77E237F3C12112C121495EE900102F078
:1021B900A3EFF0900102E0FEA3E0FFE4FC7D6412CE
:1021C9000141EE900102F0A3EFF012430E22E51354
:1021D900B4031F9000FBE0B50E05A3E0B50F005056
:1021E900119000FCE02432FB9000FBE03400F0A3E6
:1021F900EBF09000FBE0C0E0A3E0C0E07B027A00D6
:1022090079147D057C17785912081D15811581747B
:1022190006900014F07F027B027A0079141242932F
:10222900021D467F017B057A16792412429390019B
:1022390002E0FAA3E0BA0003B46400500990010275
:10224900E4F0A37464F0900102E0FAA3E0BA0B048D
:10225900B4B801D3400A900102740BF0A374B8F02A
:10226900E513B40120900102E0B40006A3E0B464D0
:1022790001D34011900103E0249CFB900102E0345A
:0A228900FFF0A3EBF0E513B402042C
:1022930012430E22E513B4031F900102E0B40B05B1
:1022A300A3E0B4B8005011900103E02464FB900153
:1022B30002E03400F0A3EBF0900102E0C0E0A3E001
:1022C300C0E07B027A0079147D057C1778691208D7
:1022D3001D158115817406900014F07F027B027A2C
:1022E300007914124293021D467F017B057A167909
:1022F30045124293900104E0FAA3E0BA0003B464E8
:10230300005009900104E4F0A37464F0E513B401F0
:1023130020900104E0B40006A3E0B46401D34011AB
:10232300900105E0249CFB900104E034FFF0A3EB53
:06233300F0E513B4020402
:1023390012430E22E513B4031F900104E0B5100502
:10234900A3E0B511005011900105E02464FB900150
:1023590004E03400F0A3EBF0900104E0C0E0A3E056
:10236900C0E07B027A0079147D057C177869120830
:102379001D158115817406900014F07F027B027A85
:09238900007914124293021D4672
:102392008F0CE4F50D750E01F50F751010AE0FAF31
:1023A200101243A48E118F12E4FE7F111243A4EF88
:1023B200900033F0E4FE7F121243A4EE900028F066
:1023C200A3EFF0E4FE7F131243A4EF90002AF01271
:0223D200000306
:1023D4001243218F13E50C14600E14600B14600873
:0823E400147003022BBC80E819
:1023EC00E50CB40117C00DC00E7B027A0079367D66
:1023FC00057C17787912081D15811581E50CB4023E
:10240C0017C00DC00E7B027A0079367D057C1778DB
:10241C008B12081D15811581E50CB40317C00DC076
:10242C000E7B027A0079367D057C17789D12081D8B
:10243C0015811581E513B4017EE50DB40006E50E9A
:06244C00B40001D3407151
:10245200E50E150E7002150DE50DB40006E50EB47D
:052462000001D340560B
:10246700AA0D75F004E50EC333CA33CAD5F0F88A4E
:102477000FF510AE0FAF101243A48E118F12E51097
:102487002401FFE4350FFE1243A4EF900033F0E57B
:10249700102402FFE4350FFE1243A4EE900028F04B
:1024A700A3EFF0E5102403FFE4350FFE1243A4EF7A
:0624B70090002AF08006EF
:1024BD00E4F50D750E0BE513B4020280030229A895
:1024CD00E50E640B450D700122E50CB4010280038D
:0324DD000225F9DC
:1024E000E50E2400FBE50D3455F5F0E511B5F002DD
:0F24F00080030225B7E512B5030280030225B76A
:1024FF007F017B057A1779AF124293C00DC00E7B17
:10250F00027A0079367D057C1778C012081D158177
:10251F0015817F027B027A007936124293E50EAA6B
:10252F000D75F004C333CA33CAD5F0F88A0FF5100E
:10253F00E5102401FFE4350FFE1243A4EF900106CE
:10254F00F0E5102402FFE4350FFE1243A4EE9000D5
:10255F00FBF0A3EFF0E5102403FFE4350FFE124369
:10256F00A4EF9000FDF0E5102404FFE4350FFE12F8
:10257F0043A4EE900102F0A3EFF0E5102405FFE471
:10258F00350FFE1243A4EE900104F0A3EFF0E51017
:10259F002406FFE4350FFE1243A4EE900107F0A3CB
:0825AF00EFF012430ED20422EA
:1025B70012430E7F017B057A1779D2124293C00D21
:1025C700C00E7B027A0079367D057C1778E3120806
:1025D7001D158115817F027B027A0079361242939D
:1025E700E4FE7F641242F612430E7E057FDC124240
:0C25F700F622E50CB40202800302282446
:10260300E50E2400FBE50D3455F5F0E511B5F002B8
:0F2613008003022753E512B50302800302275309
:102622007B057A1779F5126C98EF64016003022832
:012632002483
:102633007F017B057A187906124293C00DC00E7B89
:10264300027A0079367D057C18781712081D1581EA
:1026530015817F027B027A00793612429312441469
:10266300E50EAA0D75F004C333CA33CAD5F0F88A50
:102673000FF510AE0FAF10124467E5102401FFE40D
:10268300350FFE124467E5102402FFE4350FFE12F6
:102693004467E5102403FFE4350FFE124467E51099
:1026A3002404FFE4350FFE124467E5102405FFE41C
:1026B300350FFE124467E5102406FFE4350FFE12C2
:1026C3004467AE0FAF10E50E2400FDE50D3455FC55
:1026D300124376E5102401FFE4350FFE900106E076
:1026E300FD7C00124376E5102402FFE4350FFE90D3
:1026F30000FBE0FCA3E0FD124376E5102403FFE4B6
:10270300350FFE9000FDE0FD7C00124376E51024BA
:1027130004FFE4350FFE900102E0FCA3E0FD124349
:1027230076E5102405FFE4350FFE900104E0FCA3D9
:10273300E0FD124376E5102406FFE4350FFE900119
:1027430007E0FCA3E0FD12437612448A12430E22F3
:102753007F017B057A187906124293C00DC00E7B68
:10276300027A0079367D057C18781712081D1581C9
:1027730015817F027B027A00793612429312441448
:10278300E50EAA0D75F004C333CA33CAD5F0F88A2F
:102793000FF510AE0FAF10E50E2400FDE50D345517
:1027A300FC124376E5102401FFE4350FFE90010689
:1027B300E0FD7C00124376E5102402FFE4350FFEB2
:1027C3009000FBE0FCA3E0FD124376E5102403FF39
:1027D300E4350FFE9000FDE0FD7C00124376E5102A
:1027E3002404FFE4350FFE900102E0FCA3E0FD1298
:1027F3004376E5102405FFE4350FFE900104E0FC69
:10280300A3E0FD124376E5102406FFE4350FFE90A6
:102813000107E0FCA3E0FD12437612448A12430E43
:0B28230022E50CB4030280030229A888
:10282E00E50E2400FBE50D3455F5F0E511B5F0028B
:0F283E008003022903E512B50302800302290378
:10284D007B057A187929126C98EF640160030229CF
:01285D00A8D2
:10285E007F017B057A18793A124293C00DC00E7B28
:10286E00027A0079367D057C1778C012081D158115
:10287E0015817F027B027A0079361242931244143C
:10288E00E50EAA0D75F004C333CA33CAD5F0F88A23
:10289E000FF510AE0FAF10124467E5102401FFE4E0
:1028AE00350FFE124467E5102402FFE4350FFE12C9
:1028BE004467E5102403FFE4350FFE124467E5106C
:1028CE002404FFE4350FFE124467E5102405FFE4EF
:1028DE00350FFE124467E5102406FFE4350FFE1295
:1028EE004467E5102407FFE4350FFE1244671244D7
:0528FE008A12430E22C6
:102903007F017B057A18793A124293C00DC00E7B82
:10291300027A0079367D057C1778C012081D15816F
:1029230015817F027B027A00793612429312441496
:10293300E50EAA0D75F004C333CA33CAD5F0F88A7D
:102943000FF510AE0FAF10124467E5102401FFE43A
:10295300350FFE124467E5102402FFE4350FFE1223
:102963004467E5102403FFE4350FFE124467E510C6
:102973002404FFE4350FFE124467E5102405FFE449
:10298300350FFE124467E5102406FFE4350FFE12EF
:102993004467E5102407FFE4350FFE124467124431
:1029A3008A12430E22E513B403028003022A32E59E
:0B29B3000DB40005E50EB40C005074DC
:1029BE00050EE50E7002050D640C450D7006E4F56E
:1029CE000D750E01E50DB40005E50EB40B00505467
:1029DE00AA0D75F004E50EC333CA33CAD5F0F88AD2
:1029EE000FF510AE0FAF101243A48E118F12E5101B
:1029FE002401FFE4350FFE1243A4EF900033F0E5FF
:102A0E00102402FFE4350FFE1243A4EE900028F0CE
:102A1E00A3EFF0E5102403FFE4350FFE1243A4EFFD
:0C2A2E0090002AF0E50E640B450D7015B9
:102A3A007B027A0079367D057C18784B12081D7462
:102A4A0006900036F07F017B027A007936124293B3
:102A5A00E513B4040122E50E2400FBE50D3455F517
:102A6A00F0E511B5F0028003022B7FE512B50302EF
:052A7A008003022B7F28
:102A7F00900033E0601514603C1460621470030220
:0B2A8F002B16147003022B3F022B6675
:102A9A00900028E0C0E0A3E0C0E0A3E0FBE4C0E0CF
:102AAA00C0037B027A0079367D057C18785C1208AF
:102ABA001D74FC2581F581022B66900028E0C0E098
:102ACA00A3E0C0E0A3E0FBE4C0E0C0037B027A001D
:102ADA0079367D057C18786E12081D74FC2581F5FF
:102AEA00818079900028E0C0E0A3E0C0E0A3E0FB89
:102AFA00E4C0E0C0037B027A0079367D057C187851
:102B0A008012081D74FC2581F5818050900028E010
:102B1A00C0E0A3E0C0E0A3E0FBE4C0E0C0037B02A6
:102B2A007A0079367D057C18789312081D74FC2585
:102B3A0081F5818027900028E0C0E0A3E0C0E0A3EF
:102B4A00E0FBE4C0E0C0037B027A0079367D057CB5
:102B5A001878A612081D74FC2581F5819000FDE005
:092B6A00600790010CE0B4011BAE
:0C2B7300742090003CF07441A3F0800F2F
:102B7F007B027A0079367D057C1878B912081D74AE
:102B8F0006900036F0E50DB40005E50EB40B0050CD
:102B9F000E7F027B027A007936124293022C827FDB
:102BAF00027B057A1879CA1242930223D47B057AE5
:0E2BBF001879DB126C98EF64016003022C821F
:102BCD007F017B057A1879EC1242937F027B057A9F
:102BDD001879FD12429312441412442AE4FE7F64C4
:102BED001242F6E4FCFEFF7D64124376E4FE7F01A3
:102BFD0090010CE0FD7C00124376E4FE7F02900113
:102C0D0012E0FD7C00124376E4FE7F03900114E098
:102C1D00FD7C00124376E4FE7F04900115E0FD7CFF
:102C2D0000124376E4FE7F0590010FE0FCA3E0FD6A
:102C3D00124376E4FE7F06900109E0FCA3E0FD124D
:102C4D004376E4FE7F07900116E0FCA3E0FD1243FE
:102C5D0076E4FE7F0890010DE0FCA3E0FD124376C3
:102C6D00E4FE7F09900113E0FD7C001243761244CF
:082C7D008A12430E220223D447
:052C85008F0C1200039A
:102C8A001243218F0DE50C146014147003022D37C2
:0E2C9A00147003022DF6147003022E6C80E2FB
:102CA8007F017B057A19790E12429390010CE0B4EA
:102CB80001117B027A00794A7D057C19781F120878
:102CC8001D800F7B027A00794A7D057C19783012C5
:102CD800081D740690004AF07F027B027A00794A48
:0E2CE800124293E50D64016005E50DB4031181
:102CF60090010CE0B40104E4F08006740190010C2C
:0B2D0600F0E50DB402028003022EF67F
:072D1100900111E0B4011B69
:102D1800124414E4FE7F01124467E4FE7F0190012F
:102D28000CE0FD7C0012437612448A12430E227F87
:0F2D3800017B057A197941124293E50DB401151B
:102D4700900112E0B40101D34005E014F08006744D
:0A2D570003900112F0E50DB402260E
:072D6100900111E0B4011B19
:102D6800124414E4FE7F02124467E4FE7F029001DD
:102D780012E0FD7C0012437612448A12430E22E5CB
:042D88000DB403146F
:102D8C00900112E0B403005005E004F080067401D9
:102D9C00900112F0900112E0B4010F7B027A0079DD
:102DAC004A7D057C19785212081D900112E0B4027C
:102DBC000F7B027A00794A7D057C19786312081D15
:102DCC00900112E0B4030F7B027A00794A7D057CF6
:102DDC0019787412081D740690004AF07F027B0269
:102DEC007A00794A124293022C8A7F017B057A1968
:102DFC00798512429390010BE0FBE4C0E0C0037BA9
:102E0C00027A00794A7D057C1578F112081D15812E
:102E1C001581740690004AF07F027B027A00794A91
:102E2C00124293E50DB4011090010BE0B40101D3F3
:0D2E3C00400690010BE014F0E50DB4020417
:102E490012430E22E50DB403028003022EF690010F
:102E59000BE0B464004003022EF690010BE004F08D
:102E6900022C8A7F017B057A197996124293900187
:102E790014E0B401117B027A00794A7D057C197846
:102E8900A712081D800F7B027A00794A7D057C19FB
:102E990078B812081D740690004AF07F027B027A06
:102EA90000794A124293E50D64016005E50DB4030A
:012EB9001107
:102EBA00900114E0B40104E4F08006740190011456
:062ECA00F0E50DB4022644
:072ED000900111E0B4011BA9
:102ED700124414E4FE7F03124467E4FE7F0390016B
:102EE70014E0FD7C0012437612448A12430E22023C
:022EF7002C8A23
:062EF900750A011200033E
:102EFF001243218F0BE50B14600C14601C1470032C
:062F0F00022F9B022FA916
:102F1500E50AB40101D34005150A022FA9750A0572
:082F2500022FA9E50AB405041E
:042F2D001200032269
:102F3100E50A64026005E50AB40329900106E0B4DC
:052F41000101D3401F57
:102F46007F017B057A1A79511242937F027B057ABB
:102F56001A79621242937E077FD01242F68031E5DB
:0C2F66000AB40327900112E06401601F10
:102F72007F017B057A1A79511242937F027B057A8F
:102F82001A79731242937E077FD01242F68005AF00
:102F92000A122C85120003800EE50AB405005004C3
:102FA200050A8003750A01E50A14601814605814B2
:102FB20070030230671470030230D51470030231BB
:042FC20017022EFFC5
:102FC6007B027A0079727D057C1A788412081D745A
:102FD60006900072F07F017B027A007972124293AA
:102FE60090010CE0B4010E7F027B057A1A799512E6
:102FF60042930231427F027B057A1A79A6124293E6
:10300600022EFF7B027A0079727D057C1A78B71250
:10301600081D7406900072F07F017B027A007972B7
:10302600124293900112E0B4010B7F027B057A1ADB
:1030360079C8124293900112E0B4020B7F027B051D
:103046007A1A79D9124293900112E0B403028003EE
:103056000231427F027B057A1A79EA124293022EE6
:10306600FF7B027A0079727D057C1A78FB12081DB7
:103076007406900072F07F017B027A007972124228
:1030860093900106E0B40101D35008900112E06468
:103096000160117B027A0079727D057C1B780C1227
:1030A600081D801D90010BE0FBE4C0E0C0037B021D
:1030B6007A0079727D057C1578F112081D15811547
:1030C600817F027B027A007972124293022EFF7B85
:1030D600027A0079727D057C1B781D12081D740624
:1030E600900072F07F017B027A007972124293900F
:1030F6000114E0B4010D7F027B057A1B792E124282
:103106009380397F027B057A1B793F124293022E08
:10311600FF7B027A0079727D057C1B785012081DB0
:103126007406900072F07F017B027A007972124277
:0F313600937F027B057A1879CA124293022EFF0B
:103145007F017B057A1B79A51242937F027B057A65
:103155001B79B61242937E057FDC1242F67F017B16
:10316500057A1B79C71242937F027B057A1B79D8B2
:103175001242937E057FDC1242F6750801120003A8
:103185001243218F09E5091460081460161460269E
:02319500803286
:10319700E508B40101D340041508802675080780A7
:0631A70021E508B4070455
:0431AD0012000322E7
:1031B100AF081234D4120003800EE508B4070050A2
:1031C1000405088003750801E508B4040302331EF1
:1031D1005011E50814602314606B1470030232B2BD
:1031E1000234D1E50824FB70030233691470030231
:0A31F10034091470030234A6808A2A
:1031FB007B027A00799A7D057C1B78E912081D7495
:10320B000690009AF07F017B027A00799A12429322
:10321B00900109E0C0E0A3E0C0E07B027A00799A5C
:10322B007D057C1B78FA12081D158115817F027BA9
:10323B00027A00799A1242930231857B027A0079E5
:10324B009A7D057C1C780A12081D740690009AF072
:10325B007F017B027A00799A124293E4FCFD900184
:10326B000FE0FEA3E0FF121491C004C005C006C01E
:10327B00077C6F7D127E837F3A12112CC004C00530
:10328B00C006C0077B027A00799A7D057C1C781BEF
:10329B0012081D74FC2581F5817F027B027A00796F
:1032AB009A1242930231857B027A00799A7D057CD2
:1032BB001C782D12081D740690009AF07F017B027A
:1032CB007A00799A124293E4FCFD90010DE0FEA383
:1032DB00E0FF121491C004C005C006C0077C6F7DCF
:1032EB00127E837F3A12112CC004C005C006C007A2
:1032FB007B027A00799A7D057C1C781B12081D7461
:10330B00FC2581F5817F027B027A00799A12429328
:10331B000231857B027A00799A7D057C1C783E12FE
:10332B00081D740690009AF07F017B027A00799A4F
:10333B00124293900113E0FBE4C0E0C0037B027ADE
:10334B0000799A7D057C1C784F12081D158115811B
:10335B007F027B027A00799A1242930231857B02BB
:10336B007A00799A7D057C1C786212081D74069090
:10337B00009AF07F017B027A00799A1242939001B6
:10338B0016E0FEA3E0FFE4FCFD121491C004C0059F
:10339B00C006C00774CDFC14FDFE743DFF12112C4A
:1033AB008C0A8D0B8E0C8F0D900115E0FF1245864C
:1033BB00E4FCFD121491C004C005C006C007AC0AA2
:1033CB00AD0BAE0CAF0D121288C004C005C006C009
:1033DB0007900115E0FBE4C0E0C0037B027A0079A3
:1033EB009A7D057C1C787312081D74FA2581F58172
:1033FB007F027B027A00799A1242930231857B021B
:10340B007A00799A7D057C1C788612081D740690CB
:10341B00009AF07F017B027A00799A124293900115
:10342B0016E0FEA3E0FFE4FCFD121491C004C005FE
:10343B00C006C00774CDFC14FDFE743DFF12112CA9
:06344B008C0A8D0B8E0CB3
:103451008F0D7F05124586E4FCFD121491C004C056
:1034610005C006C007AC0AAD0BAE0CAF0D12128839
:10347100C004C005C006C007900116E0C0E0A3E08B
:10348100C0E07B027A00799A7D057C1C789712084E
:103491001D74FA2581F5817F027B027A00799A12E7
:1034A10042930231857B027A00799A7D057C1C78F2
:1034B100A712081D740690009AF07F017B027A0022
:1034C100799A1242937F027B057A1879CA12429344
:0334D10002318540
:0534D4008F0E12000341
:1034D9001243218F0FE50EB404030237785014E527
:1034E9000E1460201470030235C414700302369E52
:1034F9000239EAE50E24FB70030238101470030246
:0435090038F680CC44
:10350D007F017B057A1C79B8124293900109E0C0C6
:10351D00E0A3E0C0E07B027A0079AE7D057C1B78EC
:10352D00FA12081D1581158174069000AEF07F0208
:10353D007B027A0079AE124293E50FB4011E900121
:10354D0009E0B40406A3E0B4B001D3400F90010A22
:10355D00E014F0F49001097003E014F0E50FB402EB
:01356D002736
:07356E00900111E0B4011C03
:10357500124414E4FE7F06124467E4FE7F069001C0
:1035850009E0FCA3E0FD12437612448A12430E22A1
:10359500E50FB4030280030239EA900109E0B4079C
:1035A50005A3E0B4D00040030239EA90010AE00423
:1035B500F090010960030239EAE004F00234D97F92
:1035C500017B057A1C79C912429390010FE0FEA395
:1035D500E0FFE4FCFD121491C004C005C006C0075D
:1035E5007C6F7D127E837F3A12112CC004C005C00A
:1035F50006C0077B027A0079AE7D057C1C78DA125D
:10360500081D74FC2581F58174069000AEF07F02DB
:103615007B027A0079AE124293E50FB40120900146
:103625000FE0B40606A3E0B44001D34011900110A9
:10363500E024F6FB90010FE034FFF0A3EBF0E50F7B
:03364500B40227A5
:07364800900111E0B4011C28
:10364F00124414E4FE7F05124467E4FE7F059001E7
:10365F000FE0FCA3E0FD12437612448A12430E22C0
:10366F00E50FB4030280030239EA90010FE0B407BB
:10367F0005A3E0B46C0040030239EA900110E02486
:10368F000AFB90010FE03400F0A3EBF00234D97F76
:10369F00017B057A1C79EB12429390010DE0FEA39A
:1036AF00E0FFE4FCFD121491C004C005C006C00782
:1036BF007C6F7D127E837F3A12112CC004C005C02F
:1036CF0006C0077B027A0079AE7D057C1C78DA1282
:1036DF00081D74FC2581F58174069000AEF07F0201
:1036EF007B027A0079AE124293E50FB4012090016C
:1036FF000DE0B40106A3E0B4F401D3401190010E24
:10370F00E024F6FB90010DE034FFF0A3EBF0E50FA2
:03371F00B40227CA
:07372200900111E0B4011C4D
:10372900124414E4FE7F08124467E4FE7F08900106
:103739000DE0FCA3E0FD12437612448A12430E22E7
:10374900E50FB4030280030239EA90010DE0B404E5
:1037590005A3E0B4B00040030239EA90010EE02469
:103769000AFB90010DE03400F0A3EBF00234D97F9D
:10377900017B057A1C79FC124293900113E0FBE46A
:10378900C0E0C0037B027A0079AE7D057C1D780D0F
:1037990012081D1581158174069000AEF07F027B19
:1037A900027A0079AE124293E50FB4011090011329
:1037B900E0B40501D34006900113E014F0E50FB41D
:0237C9000226D6
:0737CB00900111E0B4011BA5
:1037D200124414E4FE7F09124467E4FE7F0990015B
:1037E20013E0FD7C0012437612448A12430E22E556
:1037F2000FB4030280030239EA900113E0B4190006
:1038020040030239EA900113E004F00234D97F0147
:103812007B057A1D791F124293900116E0FEA3E008
:10382200FFE4FCFD121491C004C005C006C0077479
:10383200CDFC14FDFE743DFF12112C9000C212004B
:10384200E3900115E0FF124586E4FCFD121491C0DD
:1038520004C005C006C0079000C2121285C004C091
:1038620005C006C007900115E0FBE4C0E0C0037B81
:10387200027A0079AE7D057C1C787312081D74FAF9
:103882002581F58174069000AEF07F027B027A00FA
:1038920079AE124293E50FB40110900115E0B40025
:0F38A20001D34006900115E014F0E50FB40226A3
:0738B100900111E0B4011BBE
:1038B800124414E4FE7F04124467E4FE7F0490017E
:1038C80015E0FD7C0012437612448A12430E22E56D
:1038D8000FB4030280030239EA900115E0B4040032
:1038E80040030239EA900115E004F00234D97F015F
:1038F8007B057A1D7930124293900116E0FEA3E011
:10390800FFE4FCFD121491C004C005C006C0077492
:10391800CDFC14FDFE743DFF12112C9000C2120064
:10392800E37F05124586E4FCFD121491C004C0052E
:10393800C006C0079000C2121285C004C005C006A8
:10394800C007900116E0C0E0A3E0C0E07B027A0067
:1039580079AE7D057C1C789712081D74FA2581F5CF
:103968008174069000AEF07F027B027A0079AE1275
:103978004293E50FB4011E900116E0B40706A3E0D8
:10398800B4D001D3400F900117E014F0F490011661
:0A3998007003E014F0E50FB40227FD
:0739A200900111E0B4011CCB
:1039A900124414E4FE7F07124467E4FE7F07900186
:1039B90016E0FCA3E0FD12437612448A12430E225C
:1039C900E50FB4031C900116E0B40B05A3E0B4B8ED
:1039D90000500E900117E004F09001167003E00406
:0439E900F00234D9DB
:1039ED002053746172742043686172676572202080
:1039FD0000202020202020202020202020202532C3
:103A0D00642000205374617274204469736368618B
:043A1D007267650067
:103A21008E088F098D0A8D07123FEAEE9000E6F0AD
:103A3100A3EFF0E4FDFC9000DAF0900116E0FEA3A4
:103A4100E0FF1214919000DC1200E3E4FCFD900110
:103A510007E0FEA3E0FF121491C004C005C006C038
:103A6100077C6F7D127E837F3A12112CC004C00542
:103A7100C006C0079000FDE0FF7E00E433E4500182
:103A810014FCFD12145412112CC004C005C006C050
:103A9100079000DC121129121495EE9000E2F0A3B8
:103AA100EFF0E50A24FD7003023CE2147003023CCE
:093AB100E224FE6004146001220D
:103ABA00AF0A123FEAEE9000E0F0A3EFF070189020
:103ACA0000E0E070129000E6E0FAA3E0FB9000E06C
:103ADA00EAF0A3EBF080109000E0E0FAA3E0FB909C
:103AEA0000E6EAF0A3EBF0E4FCFDAE08AF0912141D
:103AFA0091C004C005C006C0077C297D5C7E0F7F8B
:103B0A003D12112C121495EE9000E4F0A3EFF0E5AB
:093B1A000AB406028003023BA874
:0E3B23009000DBE0F5F0900119E065F06077AE
:103B3100E09000DBF07B027A0079C67D057C397864
:103B4100ED12081D74069000C6F07F017B027A0019
:103B510079C6124293E5FEFF7E00E4FC7D6412010A
:103B610041E4FC7DFF120155C006C0077B027A00CB
:103B710079C67D057C3978FE12081D158115818570
:103B8100080B85090C7B027A0079C69000E0E0FC05
:103B9100A3E0FD12404174259000D5F07F027B0225
:103BA1007A0079C61242939000E0E0FAA3E0FBEAC2
:103BB100FEEBFF9000E5E0F8E509C398FD9000E415
:103BC100E0FBE5089BFCF5F0EAB5F004EFB5050074
:103BD100500CE5FEFB7A00B4F100500205FE9000A6
:103BE100E0E0FAA3E0FB9000E5E02509FD9000E4A8
:103BF100E03508FCF5F0EAB5F005EBB50501D34079
:103C01000AE5FEB40001D3400215FE9000E0E0FC9D
:103C1100A3E0FD9000E5E0FAE509C39AFB9000E41A
:103C2100E0F8E50898FAF5F0ECB5F004EDB503001D
:103C3100401EA3E02509FB9000E4E03508FAF5F009
:103C4100ECB5F005EDB50301D350058C068D0722C7
:103C5100E5FEB40101D3400AE5FEFB7A00B4F000B1
:103C610040099000E0E0FEA3E0FF22900106E0B4ED
:053C71000101D34049F0
:103C760012402AE4FCFD121491C004C005C006C01F
:103C860007E4FCFD9000E2E0FEA3E0FF121491C001
:103C960004C005C006C0079000DC12009CE4FEFCD0
:103CA600FD743FFF12112C120FCC121522BF010911
:103CB6009000E0E0FEA3E0FF229000DAE004F0E5E9
:103CC6000AB407028003023ABAE0B40801D35003EB
:0C3CD600023ABA9000E0E0FEA3E0FF22FA
:103CE200AF0A123FEAEE9000E0F0A3EFF0701890F6
:103CF20000E0E070129000E6E0FAA3E0FB9000E042
:103D0200EAF0A3EBF080109000E0E0FAA3E0FB9071
:103D120000E6EAF0A3EBF0E4FCFDAE08AF091214F2
:103D220091C004C005C006C0077C297D5C7E0F7F60
:103D32003D12112C121495EE9000E4F0A3EFF0E581
:093D42000AB403028003023DD023
:0E3D4B009000DBE0F5F0900119E065F0607784
:103D5900E09000DBF07B027A0079C67D057C3A7839
:103D69001012081D74069000C6F07F017B027A00CC
:103D790079C6124293E5FDFF7E00E4FC7D641201E1
:103D890041E4FC7DFF120155C006C0077B027A00A1
:103D990079C67D057C3978FE12081D158115818546
:103DA900080B85090C7B027A0079C69000E0E0FCDB
:103DB900A3E0FD12404174259000D5F07F027B02FB
:103DC9007A0079C61242939000E0E0FAA3E0FB90F2
:103DD90000E5E0F8E509C398FD9000E4E0F8E5089E
:103DE90098FCF5F0EAB5F004EBB50500500CE5FDDB
:103DF900FB7A00B4F100500205FD9000E0E0FAA35F
:103E0900E0FB9000E5E02509FD9000E4E03508FCC1
:103E1900F5F0EAB5F005EBB50501D3400AE5FDB4C7
:103E29000001D3400215FD9000E0E0FCA3E0FD9005
:103E390000E5E0FAE509C39AFB9000E4E0F8E5083B
:103E490098FAF5F0ECB5F004EDB50300401EA3E0D7
:103E59002509FB9000E4E03508FAF5F0ECB5F0052A
:103E6900EDB50301D350058C068D0722E5FDB4019C
:103E790001D3400AE5FDFB7A00B4F0004009900047
:103E8900E0E0FEA3E0FF229000DAE004F0E50AB4E6
:103E990004028003023CE2E0B40801D35003023C6F
:0A3EA900E29000E0E0FEA3E0FF223B
:103EB3008E088F0912402AEE9000E8F0A3EFF0E499
:103EC300FCFD900116E0FEA3E0FF1214919000EABE
:103ED3001200E312402AEE9000EEF0A3EFF0701808
:103EE3009000EEE070129000E8E0FAA3E0FB90008F
:103EF300EEEAF0A3EBF080109000EEE0FAA3E0FB13
:103F03009000E8EAF0A3EBF09000EA12009C7C0A30
:103F13007DD77EA37F3B12112C1214959000F0EEF7
:103F2300F0A3EFF09000EEE0FCA3E0FD9000F1E0E1
:103F3300FAE509C39AFB9000F0E0F8E50898FAF572
:103F4300F0ECB5F004EDB50300500CE5FEFB7A0090
:103F5300B4F100500205FE9000EEE0FCA3E0FD90FA
:103F630000F1E02509FB9000F0E03508FAF5F0ECEC
:103F7300B5F005EDB50301D3400AE5FEB40001D366
:103F8300400215FE9000EEE0FCA3E0FD9000F1E09E
:103F9300FAE509C39AFB9000F0E0F8E50898FAF512
:103FA300F0ECB5F004EDB50300401EA3E02509FBDA
:103FB3009000F0E03508FAF5F0ECB5F005EDB50347
:103FC30001D350058C068D0722E5FE64016006E5EA
:103FD300FE64F070099000EEE0FEA3E0FF22900083
:073FE300EEE0FEA3E0FF2267
:053FEA008F0B750C00B7
:103FEF00E50B24FD601214601E24FE600514600EA4
:023FFF00801E22
:104001007F06124586227F071245862220970F7F61
:1040110006124586222096067F0712458622050C48
:09402100E50CB464C9E4FEFF22C1
:03402A00750B0013
:10402D002097067F0512458622050BE50BB464F03B
:04403D00E4FEFF227C
:104041008B0D8A0E890F8C108D11E4FCFDAE10AF23
:1040510011121491C004C005C006C007E4FCFD7430
:10406100C8FE7442FF12112CC004C005C006C0076F
:10407100E4FCFDAE0BAF0C121491121288121495D0
:104081008F12AD0DAC0EA80FAB0DAA0EA90FE41245
:04409100002A7F0181
:1040950008E870010CEDFBECFAE8F9740112002A4E
:1040A5000FBF09EC08E870010CEDFBECFAE8F974B8
:0740B5000212002A7513003E
:1040BC00AF137E00E4FC7D0A1201418EF0B2F7745E
:0C40CC0080B5F006E512B50701D34041B5
:1040D800AB0DAA0EA90F740312002A050FE50F7085
:1040E80002050EE513B40800500CAB0DAA0EA90F7B
:1040F800E412002A800BAB0DAA0EA90F740312005C
:104108002AE513B4090BAB0DAA0EA90F74201200EF
:094118002A0513E513B40A9C22E8
:0A41210075D90275E90075F9002256
:10412B0075FA0075EA0075DA0075FB0075EB007522
:10413B00DB0075FC0075EC0075DC0075FD0075EDA2
:10414B000075DD0075FE0075EE0075DE00C2DED277
:0A415B0093D294D295D296D2972207
:0B416500EEB40005EFB40001D34007EA
:08417000EF1F70F11E80EE222A
:10417800C283E4FE7F641241657F331241E07F32DF
:104188001241E07F281241E07F0C1241E07F0612C5
:0F41980041E07F011241E07E017FF41241652278
:1041A7008F0553800FED54F04280D283E4FE7F32B7
:1041B700124165C28353800FEDC454F04280D2830D
:1041C700E4FE7F32124165C2837E017FF4124165AE
:0141D70022C5
:0841D8008F1FD2821241A722C1
:0841E0008F1FC2821241A722C9
:1041E8000E1F111111111F000E1F1111111F1F0099
:1041F8000E1F11111F1F1F000E1F111F1F1F1F0051
:104208000E1F1F1F1F1F1F000002060E06020000C0
:1042180000080C0E0C080000001F1517111F0000E5
:10422800001F10101010101F001F00000000001FBA
:10423800001F01010101011F001F1F1F1F1F1F1F5A
:104248000E1F11111F1F1F000002060E060200009C
:1042580000080C0E0C080000001F1517111F0000A5
:104268008F08750940E50875F040A4F508750A003F
:10427800AF091241E0E508250A9041E893FF124191
:0B428800D80509050AE50AB440E6224B
:104293008F1A8B1B8A1C891DEF14600A14600E147D
:0642A300601214601622F7
:1042A9007F801241E080137FC01241E0800C7FFFC4
:0D42B9001241E080057FFF1241E0751E00FC
:1042C600AB1BAA1CA91D120071FF1241D8051DE5E2
:0D42D6001D7002051C051EE51EB410E4223B
:0742E300900114E0B4010B8F
:0C42EA00C2B5E4FE7F3C1242F6D2B522C1
:0442F600EE4F601314
:1042FA007B007A06DBFEDAFC7C06E4FDEF1F70EC3D
:04430A001E80E92206
:07430E00900114E0B4010B63
:0C431500C2B57E037FE81242F6D2B5224A
:10432100E4F51A208003751A01208103751A022011
:104331008006208103751A03E51A60031242E330F7
:05434100800320812132
:10434600E4FE7F321242F6E523B40F01D3400EE5B8
:044356001AB402068D
:10435A00E4F5237F0422AF1A22052380D9E4F5234A
:03436A00AF1A2265
:09436D00C2A3C2A2D2A1D2A02277
:104376008C148D159000F27403F0A374E8F0D2A3A8
:10438600EF2400F517EE3405F516AE16AF171244F6
:0E439600A0AE14AF151244E5124528C2A322B2
:1043A4009000F27401F0A3742CF0D2A3EF2400F572
:1043B40015EE3406F514AE14AF151244A01243CF13
:0B43C4008E168F17C2A3AE16AF172293
:0F43CF00E4F518F519F51A751B0FE51A20E731FB
:1043DE00124552A2A0E4335401751C00F51DAB1D0D
:1043EE00AA1CA81B088005C333CA33CAD8F94519BD
:1043FE00F519EA4518F518E51B151B70CE151A8030
:06440E00CAAE18AF19222E
:104414009000F27403F0A374E8F0D2A37E047FC08A
:064424001244A0C2A32215
:10442A009000F27403F0A374E8F0D2A37E047F80B4
:09443A001244A0124528C2A3227D
:104443008E218F229000F27403F0A374E8F0D2A3BC
:104453007E047F401244A0AE21AF221244E51245F0
:0444630028C2A322A6
:104467009000F27403F0A374E8F0D2A3EF2400F5F0
:1044770015EE3407F514AE14AF151244A0124528F3
:03448700C2A322AB
:10448A009000F27403F0A374E8F0D2A37E04E4FF70
:06449A001244A0C2A3229F
:0F44A0008E188F19E4F51A751B0AE51A20E733F9
:1044AF00AB19AA18E518A81B088005C313CB13CBAB
:1044BF00D8F9EB5401751C00F51D6401451C7004FF
:1044CF00D2A18002C2A1124552E51B151B70CC155B
:0644DF001A80C8C2A122F0
:0F44E5008E188F19E4F51A751B0FE51A20E733AF
:1044F400AB19AA18E518A81B088005C313CB13CB66
:10450400D8F9EB5401751C00F51D6401451C7004B9
:10451400D2A18002C2A1124552E51B151B70CC1515
:044524001A80C8220F
:10452800C2A39000F2E0FEA3E0FF12456DD2A3748F
:10453800FFFAFB20A013EA6480B48004BB0001D317
:0A4548004007EB1B70ED1A80EA2219
:10455200D2A29000F2E0FEA3E0FF12456DC2A2904B
:0B45620000F2E0FEA3E0FF12456D2216
:10456D00E4FAFB8EF0EAB5F0068FF0EBB5F00050F3
:09457D00070BEB70EE0A80EB2243
:104586008F1A9000F51200EF00000000E49000F48E
:01459600F034
:10459700E4FE7FC8124165AF1A1245EAEE9000F9B2
:1045A700F0A3EFF09000F512009CE4FCFD9000F9F9
:1045B700E0FEA3E0FF12012C9000F51200E390004B
:1045C700F4E004F0648070C875F007A31200D712F6
:1045D70001179000F9EEF0A3EFF09000F9E0FEA3C9
:0345E700E0FF22D0
:1045EA00EF441823232354F8FFD2A40000D2A700D3
:0745FA0000C2A700007E05CE
:10460100C2A4EF30E704D2A68002C2A6EFC333FFF3
:104611000000D2A40000DEE8D2A6C2A40000D2A409
:0A4621000000C2A40000E4FF7E05C3
:10462B00EFC333FF30A5034401FFD2A40000C2A4A3
:0D463B000000DEECEF540FFCE4FFFD7E08F4
:10464800EFC333FF30A5034401FFD2A40000C2A486
:0D4658000000DEECEF2DFFE43CFED2A722B7
:10466500C0E0C083C082C0D0C002C003758C87750E
:0B4675008AFF90011AE0B46400504678
:10468000E004F0900100E0FAA3E0BA0004B40001F5
:10469000D3400CE014F0F49001007003E014F090AB
:0646A000011AE0B4325FD4
:1046A600900119E070057401F08005E4900119F09D
:1046B600900118E004F0B40401D34043E4F0803FD5
:1046C600E490011AF0A3E004F0A3E0FAA3E0BA0034
:1046D60004B40001D3400CE014F0F490011C700304
:1046E600E014F0900120E0FAA3E0BA0004B400015F
:1046F600D3400CE014F0F49001207003E014F09025
:09470600011BE0B43B01D340109B
:10470F00E4F090011FE004F090011E7003E004F04C
:0D471F00D003D002D0D0D082D083D0E032C1
:10472C0020202057454C434F4D4520544F202020EE
:10473C000020534D4152542043484152474552208A
:10474C002000436F707972696768742028432920B0
:10475C004279007777772E686F6262792D72632EBB
:10476C00636F6D00202043616E2774204163636585
:10477C007373202000202053797374656D204D6570
:10478C006D6F727920002020546869732042617427
:10479C007465727920200043616E2774204469731C
:1047AC006368617267652E0020202020202532640A
:1047BC0043202534646D41680020204E6F204261F7
:1047CC0074746572792020202000202025352E322B
:1047DC0066562025352E326656730053544F5020A2
:1047EC00444953434841524745523F0020444953A2
:1047FC0043484152474520202020202000202020E3
:10480C005761697420253364207365632E00202062
:10481C0020202020202020202020202020200020AC
:10482C0020202020202020202534646D4168002584
:10483C00352E3266562025332E31664120253364C1
:10484C00730025352E3266562025332E31664120D5
:10485C002533646D0025352E326656732020505753
:10486C004D20253264200053544F50204348415270
:10487C004745523F202020002043484152474520C5
:10488C00202020202020202020002020202020203C
:10489C002020253035646D4168002046554C4C591C
:1048AC00204348415247452020200020444953438F
:1048BC00484152474520444F4E4520002055534512
:1048CC0052205445524D494E4154454400204241DA
:1048DC0054542E204F5645522D564F4C54002042C6
:1048EC0041545420444953434F4E4E4543540020A9
:1048FC004C4F5720535550504C5920564F4C540048
:10490C002025352E326656622025352E326656739A
:10491C0020002025352E326656702025352E326625
:10492C0056652000204341502E494E202534646D9D
:10493C00416820002044495343482E54494D45209A
:10494C002533646D00204348472E54494D452020A3
:10495C00202533646D002020204E6F202020202045
:07496C0020596573202000B3
:104973007580FF7590FF75A0FF75B0FFE4FE7FFAA9
:104983001242F6124178120003E4FF12426875895D
:1049930001758C87758AFFD28C75A882124121120A
:1049A300412B12436D308007208104D2008002C264
:1049B300007F017B057A47792C1242937F027B05A6
:1049C3007A47793D1242937E077FD01242F67F01E8
:1049D3007B057A47794E1242937F027B057A4779AA
:1049E3005F124293E4FEFF1243A4BE01028003025E
:0A49F3004B11BF00028003024B11BC
:1049FD007401900111F0E4FE7F011243A4EF9001C8
:104A0D000CF0E4FE7F021243A4EF900112F0E4FEDD
:104A1D007F031243A4EF900114F0E4FE7F041243D0
:104A2D00A4EF900115F0E4FE7F051243A4EE900172
:104A3D000FF0A3EFF0E4FE7F061243A4EE90010900
:104A4D00F0A3EFF0E4FE7F071243A4EE900116F001
:104A5D00A3EFF0E4FE7F081243A4EE90010DF0A346
:104A6D00EFF0E4FE7F091243A4EF900113F0E4FE92
:0B4A7D007F101243A4BE555ABF015722
:104A8800E4FE7F111243A4EF900106F0E4FE7F12CA
:104A98001243A4EE9000FBF0A3EFF0E4FE7F1312A4
:104AA80043A4EF9000FDF0E4FE7F141243A4EE90BF
:104AB8000102F0A3EFF0E4FE7F151243A4EE90018B
:104AC80004F0A3EFF0E4FE7F161243A4EE90010772
:074AD800F0A3EFF0024C77A0
:104ADF00E4900106F09000FB7403F0A374E8F07407
:104AEF0008A3F09001027403F0A374E8F0A374011B
:104AFF00F0A374F4F09001077405F0A37478F0023A
:024B0F004C77E1
:104B1100E4900106F09000FB7403F0A374E8F074D4
:104B210008A3F09001027403F0A374E8F0A37401E8
:104B3100F0A374F4F09001077405F0A37478F07495
:104B41000190010CF0900112F0900114F07404A393
:104B5100F090010F7406F0A37440F09001097406FF
:104B6100F0A37440F09001167408F0A3E4F09001F2
:104B71000D7403F0A374B6F0740F900113F0124496
:104B810014E4FE7F0A1242F6E4FEFF124467E4FDDC
:104B9100FEFF7C0112437612448AE4FEFF1243A415
:104BA100BE01028003024C48BF00028003024C4850
:104BB1007401900111F0124414E4FE7F0A1242F6CE
:104BC100E4FE7F0190010CE0FD7C00124376E4FEDF
:104BD1007F02900112E0FD7C00124376E4FE7F0328
:104BE100900114E0FD7C00124376E4FE7F04900105
:104BF10015E0FD7C00124376E4FE7F0590010FE095
:104C0100FCA3E0FD124376E4FE7F06900109E0FC7F
:104C1100A3E0FD124376E4FE7F07900116E0FCA3BA
:104C2100E0FD124376E4FE7F0890010DE0FCA3E075
:104C3100FD124376E4FE7F09900113E0FD7C001232
:074C4100437612448A802F24
:104C4800E4900111F07F017B057A47797012429355
:104C58007F027B057A47798112429312430EE4FE64
:104C68007FC81242F612430E7E027FBC1242F690B3
:104C78000115E0B40401D340037404F07E037FE817
:104C88001242F612430E120003900112E0B4010022
:104C98004007E0B40301D340067401900112F0907C
:104CA8000106E0B40101D340067402900112F090AD
:104CB8000115E0B40401D340037404F090010FE03F
:104CC800FAA3E0FBBA0603B440004009BA0704BBE4
:104CD8006C01D3400A90010F7406F0A37440F09061
:104CE8000109E0FAA3E0FBBA0403B4B0004009BA32
:104CF8000704BBD001D3400A9001097406F0A374DD
:104D080040F0900116E0FAA3E0FBBA0703B4D00024
:104D18004009BA0B04BBB801D340099001167408C6
:104D2800F0A3E4F090010DE0FAA3E0FBBA0103B4AC
:104D3800F4004009BA0404BBB001D3400A90010D45
:104D48007403F0A374B6F0900113E0B405004007B3
:104D5800E0B41901D34006740F900113F0308009B4
:104D6800208106300003123145E490011AF09001C9
:104D78001EF0A3F090011BF0D2A99000FEF0A3F062
:104D88000490010BF0C201900141F0E4FDFC900198
:104D980044F0900109E0FEA3E0FF121491C004C0A2
:104DA80005C006C0077C6F7D127E837F3A12112CE6
:104DB8009001221200E3E4FCFD900116E0FEA3E05E
:104DC800FF121491C004C005C006C00774CDFC14BE
:0E4DD800FDFE743DFF12112C9001261200E327
:104DE600124321EF90013FF0900141E0B405030228
:104DF600581C5014E01460201470030250B524FEB1
:104E060070030252B5026C95E024F97003025DFC52
:084E1600147003026A5980C800
:104E1E00D2B2D2B3D2B490013FE0B4012F30012C04
:104E2E00740190010BF07405900141F090011CE4A7
:104E3E00F0A3743CF0A3E4F0A3F090011BF09001FA
:104E4E00A2F0A3F09001A0F0A3F0808C90013FE0BF
:034E5E00B4020398
:0D4E610012071290013FE0B4035230014FE0
:084E6E00900112E064026027CC
:104E76007402900141F090011CE4F0A3743CF0A38D
:104E8600E4F0A3F090011BF09001A2F0A3F09001D2
:074E9600A0F0A3F0026C95EF
:104E9D007F017B057A4779921242937F027B057AD7
:104EAD004779A31242937E077FD01242F6024DE658
:104EBD007F05124586EE90014EF0A3EFF090010CA8
:094ECD00E0B401028003024F93DE
:104ED600900106E0600F14600C14604214603F14E9
:054EE6006075024F930E
:104EEB00E4FCFD90014EE0FEA3E0FF121491C00420
:104EFB00C005C006C007900126121285C004C0056C
:104F0B00C006C0077455FEFCFD743FFF12112C1236
:104F1B001495EF9000FDF0806FE4FCFD90014EE0E6
:104F2B00FEA3E0FF121491C004C005C006C0079099
:104F3B000126121285C004C005C006C0077CDD7DAA
:104F4B00607E8A7F3E12112C121495EF9000FDF0BB
:104F5B008036E4FCFD90014EE0FEA3E0FF121491BD
:104F6B00C004C005C006C007900126121285C004FC
:104F7B00C005C006C007E4FEFCFD743FFF12112CF8
:104F8B00121495EF9000FDF09000FBE0C0E0A3E061
:104F9B00C0E0A3E0FBE4C0E0C0037B027A01792A06
:104FAB007D057C4778B412081D74FC2581F5819032
:104FBB0000FDE070067441900130F07B027A0179BC
:104FCB002A900106E0FD126D307F017B027A017998
:104FDB002A124293900115E0FF124586EE9001A62E
:104FEB00F0A3EFF0E4FCFD90014EE0FEA3E0FF1216
:104FFB001491C004C005C006C0079001261212858B
:10500B00C004C005C006C0077466FEFCFD743FFFFC
:0E501B00121522BFFF0280069000FDE0701902
:105029007B027A01792A7D057C4778C512081D74AF
:095039000690012AF0C201806515
:10504200E4FCFD9001A6E0FEA3E0FF121491C0046F
:10505200C005C006C007900126121285C004C00513
:10506200C006C007E4FCFD90014EE0FEA3E0FF1283
:105072001491C004C005C006C00790012612128513
:10508200C004C005C006C0077B027A01792A7D05EB
:105092007C4778D612081D74F82581F58174029038
:1050A200012AF0D2017F027B027A01792A1242930D
:1050B200024DE6D2B3D2B412412B7F05124586E4EB
:1050C200FCFD121491C004C005C006C00790012661
:1050D200121285C004C005C006C0077466FEFCFD3E
:0950E200743FFF121522BFFF3ECE
:1050EB00C2017408900141F0E4A3F07404A3F01220
:1050FB00412B9001A2E4F0A3F09001A0F0A3F0905B
:10510B00011CF0A37404F07F05124586EE9001A4F8
:10511B00F0A3EFF0900160E4F0A3F0024DE69001F4
:05512B003FE0B402505A
:105130007B057A4779E7126C98EF64016003026C93
:0151400095D9
:105141007F05124586EE9001A4F0A3EFF012412BEA
:1051510012430E7408900141F0E4A3F07402A3F02D
:105161009001A2E4F0A3F09001A0F0A3F090011C43
:10517100F0A37404F0900160E4F0A3F0024DE67B2B
:10518100027A01792A7D057C4778F812081D7B0295
:105191007A017935900106E0FD126D3074069001B7
:1051A1002AF07F017B027A01792A12429390011C35
:1051B100E0C0E0A3E0C0E07B027A01792A7D057CB2
:1051C10048780912081D15811581740290012AF091
:0751D100900119E0B4010A8E
:0A51D800740790012BF0C2B28002B0
:1051E200D2B27F027B027A01792A12429390011C89
:0D51F200E060030252A7A3E060030252A791
:1051FF00C2B275FD0175ED0175DD42D2DE9001225F
:10520F0012009CE4FCFD900104E0FEA3E0FF1214E9
:10521F009112112C121495EE900148F0A3EFF01299
:10522F0000037F01124268900148E0FEA3E0FF7D7A
:10523F0003123A21EE900146F0A3EFF07F027B05B7
:10524F007A48791A124293E4FF124268740490016B
:0B525F0041F0E4900144F090013EF0AB
:10526A00900146E0FCA3E0FD90013EE0FA2AFB240F
:10527A0064F582E43401F583ECF0A3EDF090014E7D
:10528A00E0FCA3E0FDEB2478F582E43401F583EC3D
:10529A00F0A3EDF090013EE004F0B40AC390011EC1
:1052AA00E4F0A3F090011BF0024DE6C2B290013F78
:1052BA00E064016004E0B403067405900144F090D0
:0652CA00013FE0B4025AAE
:1052D0007B057A4779E7126C98EF64016003026CF2
:0152E0009538
:1052E1007F05124586EE9001A4F0A3EFF012412B49
:1052F10012430E7408900141F0E4A3F07402A3F08C
:1053010090011EE0FAA3E0FB9001A2EAF0A3EBF00A
:105311009001A0E4F0A3F090011CF0A37404F090BC
:105321000160E4F0A3F0024DE690011BE0F5F0907E
:0A5331000140E065F070030254EC47
:10533B00900144E0B40001D34003E014F090011558
:10534B00E0FF124586EE9001A6F0A3EFF07F04126A
:10535B003FEAEE900174F0A3EFF09001A81200EF7A
:09536B0000000000E490013EF096
:1053740090013EE025E02466F582E43401F583E003
:10538400FCA3E0FD90013EE0FA2AFF2464F582E4E8
:105394003401F583ECF0A3EDF09001A812009CEF2A
:1053A4002464F582E43401F583E0FEA3E0FFE4FC29
:1053B400FD12012C9001A81200E390013EE004F0DC
:1053C400B408AD75F0039001A81200D7120117902C
:1053D4000146EEF0A3EFF0A3E0FEA3E0FFE4FCFD42
:1053E400121491C004C005C006C0077C297D5C7EF0
:1053F4000F7F3D12112C121495EE90015CF0A3EF77
:10540400F0900146E0FCA3E0FDA3E0FAA3E0FB90EA
:10541400015DE0F8EBC398FB90015CE0F8EA98FAD0
:10542400F5F0ECB5F004EDB50300401EE0FAA3E09E
:10543400FB900149E02BFB900148E03AFAF5F0ECCF
:0A544400B5F005EDB50301D34015E6
:10544E00900148E0FEA3E0FF7D04123A21EE9001A8
:10545E0046F0A3EFF012402AEE900188F0A3EFF091
:0F546E009001A81200EF00000000E490013EF052
:10547D0090013EE025E0247AF582E43401F583E0E5
:10548D00FCA3E0FD90013EE0FA2AFF2478F582E4CA
:10549D003401F583ECF0A3EDF09001A812009CEF20
:1054AD002478F582E43401F583E0FEA3E0FFE4FC0B
:1054BD00FD12012C9001A81200E390013EE004F0D2
:1054CD00B408AD75F0039001A81200D71201179022
:1054DD00014EEEF0A3EFF090011BE0900140F09033
:1054ED00014EE0B40006A3E0B40001D35003025511
:1054FD00E5E4FCFD90014EE0FEA3E0FF121491C027
:10550D0004C005C006C007900126121285C004C054
:10551D0005C006C0079000FDE0FB7A00E433E450BF
:10552D000114FCFDAE02AF03121454C004C005C03B
:10553D0006C007E4FCFD90010DE0FEA3E0FF121490
:10554D0091C004C005C006C0077C6F7D127E837FAD
:0D555D003A12112C12112C121522BFFF7BE7
:10556A0090014EE0FAA3E0FB9001A4EAF0A3EBF06D
:0A557A0012412B900112E0B4012948
:1055840090011CE4F0A3743CF07405900141F09088
:10559400011EE0FAA3E0FB9001A2EAF0A3EBF09075
:0955A400011EE4F0A3F0026C9575
:1055AD0012430E7408900141F0E4A3F004A3F090AF
:1055BD00011EE0FAA3E0FB9001A2EAF0A3EBF0904C
:1055CD0001A0E4F0A3F090011CF0A37404F090018D
:1055DD0060E4F0A3F0024DE6E4FCFD90014EE0FE28
:1055ED00A3E0FF121491C004C005C006C0079001CE
:1055FD0026121285C004C005C006C0077466FEFCE5
:0A560D00FD743FFF121522BFFF4C91
:1056170012412B12430E7408900141F0E4A3F07479
:1056270004A3F090011EE0FAA3E0FB9001A2EAF0C8
:10563700A3EBF09001A0E4F0A3F090011CF0A37499
:1056470004F090014EE0FAA3E0FB9001A4EAF0A376
:10565700EBF0900160E4F0A3F0024DE69000FBE070
:10566700C0E0A3E0C0E07B027A01792A7D057C488F
:10567700782B12081D158115817B027A01792D90EF
:105687000106E0FD126D30900118E0FA7404C39A28
:1056970090012AF07406A3F07F017B027A01792A30
:0C56A700124293900144E060030257B8E7
:1056B30090011EE0600302573CA3E0707C90011B45
:1056C300E0FBE4C0E0C003FCFD900146E0FEA3E084
:1056D300FF121491C004C005C006C0079001221236
:1056E3001285C004C005C006C0077C6F7D127E838F
:1056F3007F3A12112CC004C005C006C007E4FCFDAC
:1057030090014EE0FEA3E0FF121491C004C005C057
:1057130006C007900126121285C004C005C006C04A
:10572300077B027A01792A7D057C48783B12081DA4
:1057330074F62581F58102580E90011EE0C0E0A3A6
:10574300E0C0E0E4FCFD900146E0FEA3E0FF12149C
:1057530091C004C005C006C007900122121285C083
:1057630004C005C006C0077C6F7D127E837F3A129A
:10577300112CC004C005C006C007E4FCFD90014E17
:10578300E0FEA3E0FF121491C004C005C006C007E9
:10579300900126121285C004C005C006C0077B0213
:1057A3007A01792A7D057C48784E12081D74F62506
:0557B30081F581805624
:1057B800E5FDFF7E00E4FC7D64120141E4FC7DFF11
:1057C800120155C006C007E4FCFD9001A6E0FEA347
:1057D800E0FF121491C004C005C006C0079001265E
:1057E800121285C004C005C006C0077B027A017981
:1057F8002A7D057C48786112081D74FA2581F58197
:105808007425900139F07F027B027A01792A1242CD
:1058180093024DE6D2B2D2B412412B7F05124586CF
:10582800E4FCFD121491C004C005C006C007900135
:1058380026121285C004C005C006C0077466FEFCA7
:0A584800FD743FFF121522BFFF3E62
:1058520012412B12430EC2017408900141F0E4A3DD
:10586200F07404A3F09001A0E4F0A3F090011CF006
:10587200A37404F090014EE0FAA3E0FB9001A4EAC5
:10588200F0A3EBF0900160E4F0A3F0024DE690018A
:055892003FE0B4024AF2
:105897007B057A487973126C98EF64016003026C98
:0158A700956B
:1058A8007F05124586EE9001A4F0A3EFF012412B7C
:1058B80012430E7408900141F0E4A3F07402A3F0BF
:1058C8009001A0E4F0A3F090011CF0A37404F09000
:1058D8000160E4F0A3F0024DE67B027A01792A7DAB
:1058E800057C48788412081D7B027A017932900180
:1058F80006E0FD126D30740690012AF07F017B02EC
:105908007A01792A12429390011CE0C0E0A3E0C01A
:10591800E07B027A01792A7D057C48780912081D06
:1059280015811581740290012AF0900119E0B401E3
:015938000A64
:0A593900740790012BF0C2B3800246
:10594300D2B37F027B027A01792A12429390011C1F
:0D595300E06003025DEEA3E06003025DEE84
:1059600090012212009CE4FCFD74A0FE7441FF1221
:10597000112C121495EE900152F0A3EFF0E4FCFD0F
:1059800090010FE0FEA3E0FF121491C004C005C017
:1059900006C0077C6F7D127E837F3A12112CC004F3
:1059A000C005C006C0079000FDE0FF7E00E433E4C0
:1059B000500114FCFD12145412112CC004C005C077
:1059C00006C007900126121129121495EE90015677
:1059D000F0A3EFF0900113E0FF7E00E433E4500108
:1059E00014FCFD121454C004C005C006C0077C6F2F
:1059F0007D127E837F3A12112CC004C005C006C000
:105A0000079000FDE0FDFFE4FE33E4500114FDFCCF
:105A100012145412112CC004C005C006C007900116
:105A200026121129121495EE900158F0A3EFF09070
:105A30000107E0FEA3E0FFE4FCFD121491C004C0E6
:105A400005C006C0077C6F7D127E837F3A12112C41
:105A5000C004C005C006C0079000FDE0FD7C00E466
:105A6000C0E0EDFFD0E0FE33E4500114FDFC121461
:105A70005412112CC004C005C006C00790012612A4
:105A80001129121495EE90014CF0A3EFF09000FB59
:105A9000E0FEA3E0FF900102E0FCA3E0FD12017D27
:105AA000E4FCFD121491C004C005C006C007749A3E
:105AB000FC14FDFE743FFF12112CC004C005C0068B
:105AC000C007E4FCFD7461FE7445FF12112C121432
:105AD00095EE900120F0A3EFF09000FDE0FF7E0036
:105AE000E433E4500114FCFD121454C004C005C09A
:105AF00006C0077466FCFD74B6FE743FFF12112CDD
:105B0000C004C005C006C007900126121129121456
:105B100095EE90015AF0A3EFF090012612009CE45C
:105B2000FEFCFD743FFF12112C121495EE90015EE5
:105B3000F0A3EFF0900115E0B4046DE4FCFD9001DA
:105B400007E0FEA3E0FF121491C004C005C006C028
:105B5000077C6F7D127E837F3A12112CC004C00532
:105B6000C006C0079000FDE0FF7E00E433E4500172
:105B700014FCFD12145412112CC004C005C006C040
:105B800007E4FCFD7480FE743FFF120FD5C004C013
:105B900005C006C007900126121129121495EE9037
:105BA0000150F0A3EFF0801D90012612009CE4FC50
:105BB000FD7428FE7441FF12112C121495EE900111
:105BC00050F0A3EFF090012612009C7C0A7DD77E56
:105BD000237F3C12112C121495900162EEF0A3EF7A
:105BE000F0900106E0FA64026003BA032D900122EE
:105BF00012009C9000FDE0FF7E00E4FC7D3212016B
:105C000041EE33E4500114FDFC12145412112C1215
:105C10001495EE900154F0A3EFF0900106E0B40467
:105C20003A9000FBE4FCFDE0FEA3E0FF121491C0FB
:105C300004C005C006C0077C297D5C7E8F7F3D12B5
:105C4000112CC004C005C006C00790012212112902
:105C5000121495EE900154F0A3EFF0900106E0B419
:105C60000101D3404BE4FCFD900154E0FEA3E0FFB2
:105C7000121491C004C005C006C007900122120092
:105C80009CE4FCFD7448FE7442FF12112C12152294
:105C9000BFFF1D90012212009CE4FCFD7448FE74BD
:105CA00042FF12112C121495EE900154F0A3EFF064
:105CB000900106E0B40101D34006740190010BF09D
:105CC000C202E4900142F090014EE0FAA3E0FB90A2
:105CD000014AEAF0A3EBF0E4900144F0900160F097
:025CE000A3F02F
:105CE200900145F09000FEF0A3F0C0E0C0E07461C6
:105CF200C0E07445C0E0900102E0FAA3E0FBE4FCDE
:105D0200FDAE02AF03121491121288C004C005C086
:105D120006C007E4FCFD74C8FE7442FF12112C1287
:105D22001495EE900100F0A3EFF0C2B375FE017579
:105D3200EE0175DE42D2DEC20390012212009CE423
:105D4200FCFD900102E0FEA3E0FF12149112112C5F
:105D5200121495EE900148F0A3EFF01200037F01B8
:105D6200124268900148E0FEA3E0FF7D06123A214C
:105D7200EE900146F0A3EFF07F027B057A48791A94
:0D5D8200124293E4FF124268E490013EF0EB
:105D8F00900146E0FCA3E0FD90013EE0FA2AFB24DF
:105D9F0064F582E43401F583ECF0A3EDF090014E4D
:105DAF00E0FCA3E0FDEB2478F582E43401F583EC0D
:105DBF00F0A3EDF0900115E0FF12458690013EE053
:105DCF00FA2A248CF582E43401F583EEF0A3EFF088
:105DDF0090013EE004F0B40AA77407900141F090DF
:105DEF00011EE4F0A3F090011BF0024DE6C2B39048
:105DFF00013FE064016004E0B403067405900144C0
:0B5E0F00F0900100E0705DA3E070590E
:105E1A009000FFE004F09000FE7003E004F0E4C09C
:105E2A00E0C0E07461C0E07445C0E0E4FCFD9001AC
:105E3A0046E0FEA3E0FF121491C004C005C006C0EC
:105E4A0007900122121285121288C004C005C006EA
:105E5A00C007E4FCFD74C8FE7442FF12112C121430
:105E6A0095EE900100F0A3EFF0900120E0600302AC
:095E7A005F04A3E06003025F0471
:0A5E830090010BE0B40101D340369A
:105E8D001242E390010BE014F07402900141F01204
:105E9D00412B90011CE4F0A3743CF0A3E4F0A3F0BB
:105EAD0090011BF09001A2F0A3F09001A0F0A3F0DF
:105EBD001242E3024DE612412B12430E740890017B
:105ECD0041F0E4A3F0A3F090011EE0FAA3E0FB90F3
:105EDD0001A0EAF0A3EBF090011CE4F0A37404F030
:105EED0090014EE0FAA3E0FB9001A4EAF0A3EBF0E1
:0E5EFD00900160E4F0A3F090013FE0B4025A7F
:0E5F0B007B057A487973126C98EF6401704C34
:105F190012412B12430E740190010BF07408900189
:105F290041F0E4A3F07402A3F090011EE0FAA3E0AB
:105F3900FB9001A0EAF0A3EBF090011CE4F0A3743C
:105F490004F090014EE0FAA3E0FB9001A4EAF0A36B
:105F5900EBF0900160E4F0A3F0024DE63003030298
:025F69006120B5
:105F6B0090011BE0F5F0900140E065F070030262D8
:015F7B00FB2A
:105F7C00900144E0B40001D34003E014F07F071219
:105F8C003FEAEE900174F0A3EFF09001A81200EF3D
:095F9C0000000000E490013EF059
:105FA50090013EE025E02466F582E43401F583E0C6
:105FB500FCA3E0FD90013EE0FA2AFF2464F582E4AB
:105FC5003401F583ECF0A3EDF09001A812009CEFED
:105FD5002464F582E43401F583E0FEA3E0FFE4FCEC
:105FE500FD12012C9001A81200E390013EE004F09F
:105FF500B408AD75F0039001A81200D712011790EF
:106005000146EEF0A3EFF0A3E0FEA3E0FFE4FCFD04
:10601500121491C004C005C006C0077C297D5C7EB2
:106025000F7F3D12112C121495EE90015CF0A3EF39
:10603500F0900146E0FCA3E0FDA3E0FAA3E0FB90AD
:10604500015DE0F8EBC398FB90015CE0F8EA98FA93
:10605500F5F0ECB5F004EDB50300401EE0FAA3E061
:10606500FB900149E02BFB900148E03AFAF5F0EC92
:0A607500B5F005EDB50301D34015A9
:10607F00900148E0FEA3E0FF7D07123A21EE900168
:10608F0046F0A3EFF012402AEE900188F0A3EFF054
:0F609F009001A81200EF00000000E490013EF015
:1060AE0090013EE025E0247AF582E43401F583E0A8
:1060BE00FCA3E0FD90013EE0FA2AFF2478F582E48D
:1060CE003401F583ECF0A3EDF09001A812009CEFE3
:1060DE002478F582E43401F583E0FEA3E0FFE4FCCE
:1060EE00FD12012C9001A81200E390013EE004F095
:1060FE00B408AD75F0039001A81200D712011790E5
:10610E00014EEEF0A3EFF090011BE0900140F00283
:02611E0062FB22
:1061200090011BE0F5F0900140E065F07003026221
:01613000FB73
:10613100900144E0B40001D34003E014F012402A7E
:10614100EE900188F0A3EFF09001A81200EF00009B
:076151000000E490013EF0A4
:1061580090013EE025E0247AF582E43401F583E0FD
:10616800FEA3E0FF90013EE0FA2AFD7C002478F5CA
:1061780082E43401F583EEF0A3EFF09001A8120059
:106188009CED2478F582E43401F583E0FEA3E0FF7A
:10619800E4FD12012C9001A81200E390013EE004F6
:1061A800F0B408AC75F0039001A81200D7120117DB
:1061B80090014EEEF0A3EFF0900106E0B4042EE457
:1061C800FCFD90014CE0FEA3E0FF121491C004C056
:1061D80005C006C0077C297D5C7E0F7F3D12112C0F
:1061E800121495EE90015CF0A3EFF0801C9001264C
:1061F80012009C7C0A7DD77EA37F3B12112C1214BF
:1062080095EE90015CF0A3EFF090014EE0FCA3E066
:10621800FD90014CE0FAA3E0FB90015DE0F8EBC3D0
:1062280098FB90015CE0F8EA98FAF5F0ECB5F00418
:10623800EDB50300401EE0FAA3E0FB90014DE02B12
:10624800FB90014CE03AFAF5F0ECB5F005EDB5033A
:0462580001D340131B
:10625C0090014CE0FEA3E0FF123EB3EE90014EF035
:10626C00A3EFF07F07123FEAEE900174F0A3EFF07A
:0F627C009001A81200EF00000000E490013EF036
:10628B0090013EE025E02466F582E43401F583E0DD
:10629B00FEA3E0FF90013EE0FA2AFD7C002464F5AA
:1062AB0082E43401F583EEF0A3EFF09001A8120025
:1062BB009CED2464F582E43401F583E0FEA3E0FF5A
:1062CB00E4FD12012C9001A81200E390013EE004C2
:1062DB00F0B408AC75F0039001A81200D7120117A7
:1062EB00900146EEF0A3EFF090011BE0900140F01F
:1062FB00900106E06004E0B40172900152E0FAF5FF
:10630B00F0A3E0FB900146E0B5F006A3E0B5030176
:03631B00D3505903
:10631E007F05124586EE9001A4F0A3EFF012412BFB
:10632E0075FD7F75ED7F75DD42D2DE12430E740171
:10633E0090010BF0C2017408900141F0E4A3F074D7
:10634E0004A3F090011EE0FAA3E0FB9001A0EAF096
:10635E00A3EBF090011CE4F0A37404F0900160E450
:10636E00F0A3F012412B024DE6900106E0FAB401C3
:10637E0001D35003026421900152E0FCA3E0FD9092
:10638E000146E0B50406A3E0B50501D3400302645F
:10639E002190014EE0FEA3E0FF90015EE0FCA3E041
:1063AE00FD90014DE02DFD90014CE03CFCF5F0EE32
:0A63BE00B5F005EFB50501D3405915
:1063C8007F05124586EE9001A4F0A3EFF012412B51
:1063D80075FD7F75ED7F75DD42D2DE12430E7401C7
:1063E80090010BF0C2017408900141F0E4A3F0742D
:1063F80004A3F090011EE0FAA3E0FB9001A0EAF0EC
:10640800A3EBF090011CE4F0A37404F0900160E4A5
:10641800F0A3F012412B024DE6900106E06004E083
:03642800B401506C
:10642B00900156E0FAA3E0FB90014EE0B50206A303
:07643B00E0B50301D3403975
:106442007F05124586EE9001A4F0A3EFF012412BD6
:1064520012430E7408900141F0E4A3F07403A3F018
:1064620090011EE0FAA3E0FB9001A0EAF0A3EBF09A
:1064720090011CE4F0A37404F0900106E06009E0CE
:10648200B4010280030265A990015AE0FAF5F0A373
:10649200E0FB90014EE0B5F006A3E0B50301D35056
:0464A200030265A9E3
:1064A600900160E0FAA3E0FB90014EE0B50206A37E
:0764B600E0B50301D3401E15
:1064BD0090014EE0FAA3E0FB900160EAF0A3EBF04F
:0E64CD00900106E060030265A9C2020265A903
:1064DB00900159E0FB900158E0C313CB13CBFA901A
:1064EB000160E0FCA3E0FD90014FE0F8EDC398FDE7
:1064FB0090014EE0F8EC98B50205EDB50301D340E1
:10650B0002D202900158E0FCA3E0FD900160E0FA9A
:10651B00A3E0FB90014FE0F8EBC398FB90014EE03A
:0D652B00F8EA98B50405EBB50501D3407101
:0A65380090010BE0B40101D3402DE7
:10654200E014F07402900141F012412B90011CE41E
:10655200F0A3743CF0A3E4F0A3F090011BF09001CF
:10656200A2F0A3F09001A0F0A3F0024DE612412B9D
:1065720012430E7408900141F0E4A3F0A3F09001DD
:106582001EE0FAA3E0FB9001A0EAF0A3EBF0900179
:106592001CE4F0A37404F090014EE0FAA3E0FB9037
:1065A20001A4EAF0A3EBF0900106E0FAB401028044
:1065B200030266C490015AE0FCF5F0A3E0FD9001ED
:1065C2004EE0B5F006A3E0B50501D350030266C460
:1065D20090011CE060030266C4A3E060030266C48B
:1065E200900162E0C0E0A3E0C0E090014AE0FAA3BB
:1065F200E0FB90014FE0F8EBC398FF90014EE0F80A
:10660200EA98FE120212D003D0F0EEB5F004EFB514
:07661200030040030266A42F
:10661900900142E004F0B40101D34002D20290019A
:0866290042E0B40301D3407A02
:0A66310090010BE0B40101D3402DED
:10663B00E014F07402900141F012412B90011CE424
:10664B00F0A3743CF0A3E4F0A3F090011BF09001D5
:10665B00A2F0A3F09001A0F0A3F0024DE690014E42
:10666B00E0FAA3E0FB9001A4EAF0A3EBF012412BBC
:10667B0012430E7408900141F0E4A3F0A3F09001D3
:10668B001EE0FAA3E0FB9001A0EAF0A3EBF090016F
:09669B001CE4F0A37404F0800774
:1066A400C202E4900142F090011CE4F0A3743CF0B7
:1066B40090014EE0FAA3E0FB90014AEAF0A3EBF06C
:0D66C400900106E0B40101D350030267907D
:1066D10090014CE0FAA3E0FBA3E0B50205A3E0B50D
:0766E1000300401120030E2D
:1066E800D202D203900120740EF0A37410F090012E
:1066F80054E0FAA3E0FB900146E0B50205A3E0B53B
:106708000300400302679030037E900152E0FAA331
:10671800E0FB900146E0B50206A3E0B50301D340D3
:106728006790014EE0FCA3E0FD90015EE0FAA3E073
:10673800FB90014DE02BFB90014CE03AFAF5F0ECB0
:09674800B5F004EDB50300503F6B
:10675100740190010BF09001A4ECF0A3EDF0124153
:106761002B12430E7408900141F0E4A3F0A3F090C2
:10677100011EE0FAA3E0FB9001A0EAF0A3EBF09088
:10678100011CE4F0A37404F0900160E4F0A3F09024
:1067910001A81200EF00000000900115E0FF124572
:0E67A10086EE90019CF0A3EFF0E490013EF034
:1067AF0090013EE025E0248EF582E43401F583E08C
:1067BF00FEA3E0FF90013EE0FA2AFD7C00248CF559
:1067CF0082E43401F583EEF0A3EFF09001A81200FC
:1067DF009CED248CF582E43401F583E0FEA3E0FF09
:1067EF00E4FD12012C9001A81200E390013EE00499
:1067FF00F0B408AC75F0039001A81200D71201177E
:10680F009001A6EEF0A3EFF0900150E0F5F0A3E0B9
:0F681F00FB9001A6E0B5F005A3E0B50300505EC5
:0C682E00900145E004F0B40301D3405792
:10683A0012412B12430E740190010BF0740890015F
:10684A0041F0E4A3F07405A3F090011EE0FAA3E07E
:10685A00FB9001A0EAF0A3EBF090011CE4F0A37412
:10686A0004F090014EE0FAA3E0FB9001A4EAF0A341
:10687A00EBF0A3E0FAA3E0FB900160EAF0A3EBF0EF
:02688A00800587
:10688C00E4900145F09000FEE0C0E0A3E0C0E07BA6
:10689C00027A01792A7D057C48789612081D1581AB
:1068AC0015817B027A01792C900106E0FD126D3086
:0368BC0020020AAD
:0A68BF00900118E090012AF0800D0E
:1068C900900119E0B40106740490012AF07405904E
:1068D900012BF07F017B027A01792A124293900100
:0768E90044E060030269F5C1
:1068F00090011EE06003026979A3E0707C90011BA7
:10690000E0FBE4C0E0C003FCFD900146E0FEA3E034
:10691000FF121491C004C005C006C00790012212E6
:106920001285C004C005C006C0077C6F7D127E833F
:106930007F3A12112CC004C005C006C007E4FCFD5C
:1069400090014EE0FEA3E0FF121491C004C005C008
:1069500006C007900126121285C004C005C006C0FB
:10696000077B027A01792A7D057C48783B12081D55
:1069700074F62581F581026A4B90011EE0C0E0A308
:10698000E0C0E0E4FCFD900146E0FEA3E0FF12144D
:1069900091C004C005C006C007900122121285C034
:1069A00004C005C006C0077C6F7D127E837F3A124B
:1069B000112CC004C005C006C007E4FCFD90014EC8
:1069C000E0FEA3E0FF121491C004C005C006C0079A
:1069D000900126121285C004C005C006C0077B02C4
:1069E0007A01792A7D057C48784E12081D74F625B7
:0569F00081F5818056D5
:1069F500E5FEFF7E00E4FC7D64120141E4FC7DFFC1
:106A0500120155C006C007E4FCFD9001A6E0FEA3F7
:106A1500E0FF121491C004C005C006C0079001260E
:106A2500121285C004C005C006C0077B027A017931
:106A35002A7D057C48786112081D74FA2581F58147
:106A45007425900139F07F027B027A01792A12427E
:106A550093024DE6D2B2D2B3900143E0B403028073
:106A650050500BE06012146022146032807AE024EA
:086A7500FC60511460618070A7
:106A7D007B027A01792A7D057C4878A612081DD201
:106A8D00B4805D7B027A01792A7D057C4878B71246
:106A9D00081DD2B4804A7B027A01792A7D057C4893
:106AAD0078C812081DC2B480377B027A01792A7D1D
:106ABD00057C4878D912081DC2B480247B027A0166
:106ACD00792A7D057C4878EA12081DC2B480117BB5
:106ADD00027A01792A7D057C4878FB12081DC2B423
:106AED00740690012AF07F017B027A01792A124205
:0B6AFD009390011CE0701EA3E0701AD3
:106B08001242E390011CE4F0A37404F0900142E007
:106B180004F0B40401D34002E4F0900142E0601BA9
:106B2800147003026BC0147003026C1F147003020C
:0B6B38006C3E147003026C5D026C7A6E
:106B43007F05124586EE90014EF0A3EFF0900115FC
:106B5300E0FF124586EE9001A6F0A3EFF0E4FCFD02
:106B63009001A6E0FEA3E0FF121491C004C005C08B
:106B730006C007900126121285C004C005C006C0D6
:106B830007E4FCFD90014EE0FEA3E0FF121491C068
:106B930004C005C006C007900126121285C004C0B8
:106BA30005C006C0077B027A01792A7D057C4978F6
:106BB3000C12081D74F82581F581026C7AE4FCFD42
:106BC3009001A4E0FEA3E0FF121491C004C005C02D
:106BD30006C007900126121285C004C005C006C076
:106BE30007E4FCFD900160E0FEA3E0FF121491C0F6
:106BF30004C005C006C007900126121285C004C058
:106C030005C006C0077B027A01792A7D057C497895
:106C13001E12081D74F82581F581805B9000FEE04B
:106C2300C0E0A3E0C0E07B027A01792A7D057C49BC
:106C3300783012081D15811581803C9001A2E0C0B7
:106C4300E0A3E0C0E07B027A01792A7D057C4978E4
:106C53004012081D15811581801D9001A0E0C0E040
:106C6300A3E0C0E07B027A01792A7D057C49785153
:106C730012081D158115817F027B027A01792A1280
:096C8300429390013FE0B40209C4
:0C6C8C001200037401900141F0024DE67B
:106C98008B148A1589161200037F01AB14AA15A953
:106CA800161242937B027A0179AC7D057C497862A1
:106CB80012081D74069001AEF0E49001C0F0A3F034
:086CC8009001C1E06402604686
:106CD000124321EF9001C1F064016004E0B4032984
:076CE0009001C0E0B40110B7
:106CE700E4F074069001AEF074209001B6F08012C3
:106CF70074019001C0F074209001AEF07406900109
:106D0700B6F07F027B027A0179AC12429380B2908F
:056D170001C0E0FF22B5
:106D1C004E6943444E694D484C69506F4C694F4E17
:046D2C00534C412063
:0D6D30008B088A09890A8D07E49001C2F0E2
:0A6D3D009001C2E0B40216BF031378
:106D4700AB08AA09A90A744912002A050AE50A70BC
:106D5700020509EF25E025E0FE9001C2E02E906DC7
:106D67001C93AD08AC09A80A12000E050AE50A70C3
:0D6D77000205099001C2E004F0B404BA2244
:00000001FF
